:020000041100E9
:10300000002310B5294C0120636101F0F3F9402041
:103010000223FE21264A207401F072FA002835D1DD
:103020000223FF21234A207C01F06AFA00282DD1D7
:10303000214BA2899A4226D1E389204A93420ED19C
:103040001F4B204963612368002B05D1002903D061
:103050000C22200008F09CFD01F040FA10BD1A4A35
:10306000934201D00021EEE7184B194A1B689342A6
:1030700005D9C0220421207C920001F0BBFA104B3C
:1030800014496361DFE700232374EBE7CC22382087
:10309000AC219201207401F0ADFA0028F3D10E4B5F
:1030A0000E4963610E4BE381CDE7C0468863FF1F85
:1030B0009463FF1F9663FF1F5959000083050000AA
:1030C00059420011A4BC001182150000CC63FF1FFF
:1030D00087130000B0BC0011F542001198BC00112C
:1030E000AAAAFFFFF7B5164B0192C318021D0020D4
:1030F000009388235B05D3181B685C1C1AD09CB214
:10310000402C18D88D781E0CAC466746CD782D0221
:103110003D43AE4206D1019800280ED110000C703C
:10312000240A4C7003249BB20733A343D218009B9C
:103130009A42DED3FEBD4432F9E71000FAE7C046FA
:10314000FC0F0000802213B503000324019189B213
:10315000520107319B18A14304305A1A88235B059A
:10316000C3181B68591C03D190429241104016BDF0
:1031700099B2402907D80B000733A343C0189042E7
:10318000ECD30020F3E74430F9E7134B134A1B68F4
:10319000126810B5FA24934201D81A00F824104B93
:1031A000E4021B689A4210D813000E4A12689A4231
:1031B0000ED3013307D1F823DB029C4203D10A4925
:1031C000054808F06DFA200010BDFC24E402ECE78D
:1031D000FE24E402F7E7C04600C0071100D0071143
:1031E00000E0071100F00711FFFFFF7FF0B59BB073
:1031F000150004900391402A00D9A0E006AB598045
:103200001A80FFF7C2FF0400042816D9002206A97D
:10321000FFF768FF052810D906AB1B88AB420CD11D
:10322000002D07D0514B2A000499C01808F010FC5B
:10323000002802D101201BB0F0BD06AB1D8020008C
:103240000699FFF77FFF041E7BD1069B0793FFF7CC
:103250009CFF80235B01C618802307001B039E424E
:1032600001D3F826F60288235B05F31801931B6847
:10327000013302D0019808F07BFC3D49019808F029
:103280000FFA3B1D0293331D05938822029B5205C2
:103290009B181B6808935A1C3CD044219AB2009199
:1032A000402A04D80320D11D814389B2009103999B
:1032B0001B0C8B4224D0402A22D80122300008A9BE
:1032C000FFF710FF021E1BD1380008A9FFF70AFF05
:1032D0000400042831D9009A059B9B1880225201D2
:1032E000B218934240D288235B05C118009A09A8FE
:1032F00008F0D6FB1D4B009A09A9F01808F020FA37
:10330000009A029B9446634402931A4B029AFB185C
:103310009A42BAD388235B05FC18216801980139C9
:1033200008F0BEF9200008F023FC039A07AB5A808E
:1033300030000799FFF706FF0400002C03D100209E
:1033400079E70428FBD988235B05E018069908F083
:10335000A7F90323EA1C9A4300D16BE7034B0499B6
:10336000E01808F0EDF965E70424ECE7040000112B
:10337000FFFFFF7FF80F0000F7B505001400402A9B
:1033800021D8002701AE71803780FFF7FEFE0428A8
:1033900016D93A003100FFF7A5FE042810D9368867
:1033A000BC420BD0BD4209D0221CB44200D9321C11
:1033B000064B92B2C118280008F072FB30B2FEBD75
:1033C000C04300B2FBE703204042F8E704000011CD
:1033D00037B5042204000D0001A81649FFF7CCFF01
:1033E000020004280BD1019BA34208D3AB4204D0B6
:1033F000104901A80195FFF7F9FE01203EBD0E4CD2
:1034000023682000019308F0B3FB019920000139E3
:10341000019108F045F980235B01E418074B9C42B9
:10342000EED10422034901A80195FFF7DFFE002039
:10343000E4E7C0465555000000C007110000081120
:1034400030B589B008F014F910226946254808F013
:103450006FFA254B009A9A420ED1019B029A0F2BCC
:1034600033D8002101240698013B08D2002900D05E
:103470000292029B013331D10023029325E0551CB7
:10348000F2D102002100EFE710341022200004A93D
:1034900008F04EFA029B013301D1069B0293882368
:1034A00004995B05C918059B06981A03120B049131
:1034B0000592814203D02B4201D108F069FB019BA8
:1034C000013B0193019B002BDED1029B002B03D01B
:1034D000049304984168084709B030BDE025014CC9
:1034E0002D03EFE70000011150485936F7B50F4999
:1034F0000F4B0A6804001A4084235B0013430B60DF
:10350000030003271033019300252E00112008F03B
:10351000D7F9084B1B683B40AB4002351E43202DBA
:10352000F4D1019B40C4A342EED1F7BD5CF0004052
:1035300000FEFEFF64F00040802270B5AD4CAE4B43
:10354000D200002120001C6008F09AF82300AB4A4A
:1035500088331A60AA4B1A786E23002A00D01133E0
:10356000E3620A232365A74B1878A74BA0630138B1
:10357000E361C3B2032B01D810232362A34B37228C
:103580006361C823DB00A36123008C331A60082326
:1035900036210F3AE518E16323646264E967043970
:1035A000251DE96725003B26BC352E602500C0356A
:1035B0002B602500C4352A6025000636CC352E60E8
:1035C0002500083EC8352E602500D0352960210031
:1035D000D4310B602100D8310A6021000225E0318E
:1035E0000D6025004221DC35296025001B3EE435B5
:1035F0002E602500E8352B602500EC352A6022007E
:103600000525F43215602200F032116022001831D5
:103610009032116022009432136023003C229833D0
:103620001A60AF23DB002360794B2363032805D89E
:1036300008F0F6F93302353715236360962321002D
:10364000FA225B00A360E360C8332361714BFC3155
:103650009200A3640A6062626F4A704DA262732294
:10366000E2656D3A6265A2650232E5644A60022154
:10367000616696218900A166626709210022E166E0
:10368000A2676749674A684E2167E2673560032889
:1036900011D808F0C5F996089EA61023CDE70E2391
:1036A000CBE70C23C9E720001A259C3005602000D9
:1036B0000735A03005602000A83003602300FA2001
:1036C000F8338000186023006420A43318602300BE
:1036D0005F38AC33186023000338B0331860230020
:1036E000C630B433186023000020B83318602300BC
:1036F0003825FC339D604D4D5A665D644C4D9A648F
:10370000DD619625AD001D624A4D9A675D62F53D0B
:10371000FF3D9D621E25484ADD6618675867D965DA
:103720001966DA67BE23C021444A5B00E250444B6D
:103730004900635004316250C4225200A350FA235E
:10374000E4205B000432A3500432A3503D493E4ABA
:103750003E4BD1603E49800019503E49E938FF3860
:1037600019503D49043019503C491038D1613C4949
:1037700011633C4951633C4911603C49195019009F
:103780003B48F83108603B49D16582213A4A8900BB
:103790005A501A0039490832D1671A003849B432F0
:1037A00011608821374A89005A501A0036498832F8
:1037B0001160364ADA6408F01BF8012008F038F886
:1037C00070BD200014259C30056020000435A03019
:1037D00070E7200010259C30056020000335A030E4
:1037E00068E720000E259C30056020000235A030DF
:1037F00060E7C0460004FF1F6466FF1F5071FF1F93
:103800001C46FF1F4A0AFF1F3A07000080C3C90178
:103810009A02000050C300006A180000280A000045
:10382000204E000088130000F009FF1F0040001127
:1038300068100000C4090000DC05000040420F00D1
:1038400010270000FD1BFF1FFC00FF1F0000FF1FD3
:10385000252FFF1F4D32FF1FE530FF1FD91FFF1F10
:10386000F51FFF1FA121FF1F491FFF1FC528FF1FB5
:103870008D2CFF1FD918FF1FD127FF1F3925FF1FD0
:103880004525FF1F491EFF1F011FFF1FC11DFF1FF1
:10389000F7B50B0CFF270122009300233C001E000C
:1038A0001D009446019089B262469A40100008407B
:1038B00018413618B6B2FF2F02D1012E00D19FB2A7
:1038C000009802401A41AD18ADB2FF2C02D1012D73
:1038D00000D19CB20133102BE6D10320012E07D179
:1038E000012D04D1019B2401E4191C700138FEBD97
:1038F000102EFCD10238102DF9D00230F7E710B5A8
:10390000064C2378002B07D10548FFF7EFFD05484B
:10391000FFF7ECFD0123237010BDC0462566FF1F95
:103920003866FF1F2866FF1FF0B58BB00D0001231E
:103930000190102936D8FFF7E2FF00231A001B4838
:10394000C15C01335218102BFAD1023B002A29D056
:10395000174B184C1F68002306A9E25C1600FA5C9E
:1039600056405E540133102BF7D102AA07F010FE27
:103970002A0002A9019808F00BF907F041FE23681C
:103980001B18236007F03CFE63681B18636007F098
:1039900037FEA3681B18A36007F032FEE3681B180C
:1039A000E360002318000BB0F0BDC0463866FF1F6F
:1039B000BC44FF1F2866FF1F0223F0B50124594EA7
:1039C000594D3370594B2C705B6B8FB01B68552B66
:1039D00010D0082006F060FB00280BD00023210047
:1039E00000930420524A07F033FF8023DB059C62DA
:1039F000FFF726FD002006F0E7FD08F049F8FFF785
:103A00009BFD07F08DFE1F2201240021494B0EAFC4
:103A10001A70494B1C70494B1970494B19689143F6
:103A2000163A0A431A60602219689143403A0A43E1
:103A30001A6007F095FF07F0F3FEC120FF21414B0C
:103A400080001A588A431A50C52292009858884319
:103A5000BF390143995098583B4908408021C9011A
:103A60000143802099509958C0050902090A014371
:103A7000995080213548490107F05AFE032322005E
:103A8000334901940093334808F01AF82C22324944
:103A900003A808F005F803AC61782078023406F03A
:103AA00021FBBC42F8D10121002006F035FC2B4B54
:103AB0002B4A196803201140A022D2020A431A603F
:103AC0008022196892040A431A601968254A114035
:103AD000802292030A431A60234B244A934200D85F
:103AE000012008F015F807F0ABFD07F0E9FD30788C
:103AF00007F0F6FD2878C0B207F03AFD07F050FD58
:103B00000B49042007F03CFE06F02AFD00F0A2F865
:103B100000F0CAFD00F04EFE00F00CFA00200FB0DD
:103B2000F0BDC0464A0AFF1F1C46FF1F00F00040C0
:103B30003B000108480AFF1F490AFF1F680AFF1FD0
:103B4000BCF0004000E100E0FF00FFFF2046FF1F47
:103B5000A458FF1F2056FF1FC0BB001114F00040E7
:103B6000FF7FF8FFFFFF9FFF5071FF1F0080FF1FC7
:103B700070B500252849294A29484D6308CA1B0504
:103B80001B0DED188242F9D10022264B8B63264B88
:103B900008211A628022254B9205DA67244BDA68E5
:103BA0008A43DA60234A1278012A03D09A682249AC
:103BB0000A409A600121EE242048E40002686C4328
:103BC0008A430260DA6811208A43DA6007F0F0FF66
:103BD000112007F0DDFE112007F012FF184A200C1B
:103BE0000400642390420AD8FA220023D2009042B3
:103BF00005D9144B0A21C01807F0EAFEC3B2124AD5
:103C00001372124BD4801B78002B04D1104B10215F
:103C1000187807F06DFE70BD00000540880505406E
:103C200000060540FF01000000F0004004E100E054
:103C30003CF000404A0AFF1FFFDFFFFF0038004052
:103C4000B70B000030F8FFFFA063FF1FD865FF1F10
:103C5000C863FF1F002210B51100112007F060FF9C
:103C600010BD0000F8B5002301250826394F3A4C55
:103C70003B62E3681120AB43E360E368B343E36076
:103C800007F086FE112007F093FF112007F028FEB1
:103C90004023226829001343236080236268DB02EB
:103CA000134380226360A36807201343A360A368C3
:103CB0002A4A1340A3608023A2689B011343102269
:103CC000A360236C93432364236C2B4323648023DE
:103CD0005B003B62226B224B1A402263626B1A40EC
:103CE0006263A26B1A40A263E26B1340E3631D4A56
:103CF000E3681340E36006F0DFFA2900072006F0CE
:103D00000BFB8021184A1120536C0B43536407F0BE
:103D10004FFEFD21154B164A89005A508023C720BB
:103D2000626B5B0313436363E36880003343E360C8
:103D3000E368104A1D43104BE5601958114080227A
:103D400012020A431A50802292051A600B4B5E63DE
:103D5000F8BDC04600F000403CF00040FFFFDFFF30
:103D6000EFFFEFFFFFFF7FFF003800400000FF1F65
:103D7000713B0011FF00FFFF00E100E00000054083
:103D800030B503A804880B20002C0ED14968074DDC
:103D900008784978090201430A20A94205D1012186
:103DA00020001980024B1B7A137030BD192A0000C5
:103DB000A063FF1FF7B5150008AA16884A680F4FC1
:103DC00014785278120222430A24BA4214D10122F2
:103DD000DBB2019200962A0007F012FB041E0BD101
:103DE000074B1B68002B07D068782A780002104325
:103DF00042425041013098472000FEBD0229000098
:103E00002463FF1F30B5012503790400BFB02B42A6
:103E100012D00A49408806F05FFE28420CD06A465C
:103E2000074B69465B8D55801380064B60881B7A73
:103E30001371002203F016FF3FB030BD1C63FF1F5B
:103E40006042FF1FA063FF1F10B50549054806F03B
:103E5000F9FD0421044A054806F0B6FD10BDC04630
:103E60001C63FF1FFFFF0000ECBB00116042FF1F3F
:103E700010B5024804F078FD10BDC046053E0011A3
:103E8000062310B5837010330371443B43712A330A
:103E900083714433C37100230222012103720E4B4C
:103EA000027041701C8881724472197A0273C17267
:103EB0009A784273DA7882730322C2731A79027491
:103EC0005A7942740C2282749A79C274DB79037530
:103ED0001123C370152010BDA063FF1F10B514205F
:103EE00007F0F6FB124B14220021186007F080FD4A
:103EF000002007F0EDFC012007F022FD022007F072
:103F0000F7FB032003F0D4FF042005F0E9FF0520B0
:103F100003F012FA062003F0DFFE072001F0A4F8F8
:103F2000082006F031FD092000F07EFE10BDC046DD
:103F30002863FF1F10B507F0E3FD012007F050FCD8
:103F400007F006FD002010BD094B10B50400984293
:103F500005D0012904D12000064906F073FD10BDEB
:103F60000229FCD1013904F0BDFC0028F3D0F6E7AA
:103F7000FEFF00004E63FF1F70B50D7A100004AA0B
:103F80002C00168810221440154220D1002E20D17A
:103F90000A78022A18D14A68517815780E4A09021F
:103FA0002943914205D00D4A914209D01C800A2430
:103FB00004E014220A491A8007F0EAFD200070BDCF
:103FC0000C2208491A80F7E71C800124F6E7082430
:103FD000F4E70B24F2E7C046F3FF0000F4FF000013
:103FE000A044FF1FC8BC001110B5040007490848D1
:103FF00006F028FD074804F0F7FB0020E40704D58D
:104000000721054A054806F0DFFC10BD4E63FF1F7F
:10401000FFFF0000493F001130BC0011A442FF1F08
:1040200000B50C4BBFB01A780B4901A800F0F6FBA5
:104030006B4680B25880002809D06A46074B694613
:104040001B881380064B0022188803F00BFE3FB03C
:1040500000BDC0462C63FF1F2D63FF1FFE42FF1FE4
:10406000FE43FF1F00B50C4BBFB01A780B4901A8E7
:1040700001F03AFD6B4680B25880002809D06A46AC
:10408000074B69465B8D1380064B0022188803F0AE
:10409000E9FD3FB000BDC0465663FF1F5763FF1FD9
:1040A000A442FF1FFE43FF1FF7B50E00377A1C0026
:1040B00008AB11003D001A8820231D401F423CD14F
:1040C0003378022B3BD173681F785B781B023B432C
:1040D0001E4FBB4208D01E4FBB4214D01D4DAB42F9
:1040E00021D00A252800FEBD002A2AD1142C2AD866
:1040F0002200F06807F04CFD174B1C70012CF1D921
:10410000FFF7B0FFEEE7002A1BD1202C1BD82200BE
:10411000F06807F03DFD114B04211C70104B18781E
:1041200007F0E6FBDEE7E3B20124009201940A0007
:10413000310007F065F90500D4E70825D2E701252D
:10414000D0E70B25CEE70D25CCE7C046F3FF0000F6
:10415000F4FF0000022900005663FF1F2C63FF1FBD
:10416000C863FF1F70B5160004AA148805AA157845
:104170004A685078117800022A4A084380180528B6
:104180004BD807F04DFC03131E29343F0720032CA6
:104190000BD80422121BAA4200D92A0022491A80F5
:1041A0003000091907F0F4FC002070BD0720112C25
:1041B000FBD81222121BAA4200D92A001B491A80DE
:1041C000EEE707200E2CF0D80F22121BAA4200D9CE
:1041D0002A0017491A80E3E70720032CE5D80422B8
:1041E000121BAA4200D92A0012491A80D8E70720D8
:1041F000032CDAD80422121BAA4200D92A000E4945
:104200001A80CDE70720032CCFD80422121BAA4224
:1042100000D92A0009491A80C2E700220A201A8020
:10422000C3E7C046DCD5FFFF7BBC00117463FF1FF2
:104230006BBC001166BC001161BC00115CBC0011BC
:1042400010B50D21024A034806F0BEFB10BDC04662
:1042500050BC00111443FF1F37B5002000F0CAF80E
:10426000204D214BEA89287C9A422AD1042201A9B7
:1042700000F074F9040000F031F9002C30D16B46E5
:1042800099882B68C9BA4B432989184A1B145B18B3
:1042900053806B46D9886B6849BA89B24B436989A8
:1042A0001B0C5B181248191C1BB2834200DD011C59
:1042B0000B0400D500211388918001331380200066
:1042C0003EBD0223002101AA00F01AF96A4604004B
:1042D00002230121287C063200F012F90443CAE7C8
:1042E0000124ECE78863FF1F83050000A063FF1F24
:1042F0000F27000037B5012000F07CF81E4D072283
:104300006946287C00F02AF9041E31D16B461B78DF
:104310007F2B2DD800F0E2F86B46D878F02302040A
:104320001B031A406B469B8814495BBA9BB21A4325
:104330002B68000953432A891B0C9B184B806B4642
:104340005A789B7812031B011A436B68024353434C
:104350006A891B0C9B181AB21B0402D58C802000A2
:104360003EBD074B9A4201DC8A80F8E78B80F6E776
:1043700000F0B4F80124F2E78863FF1FA063FF1F79
:104380000F27000010B50F4C237C002B0CD0382BCE
:104390000BD1012000F02EF8CC22AC21207C920120
:1043A00000F028F900F09AF810BD074BE2899A4214
:1043B000FAD1012000F01EF80021207C00F0FAF86C
:1043C000F0E7C0468863FF1F8305000010B5084B67
:1043D0001A7C002A09D05B69002B06D09847041E7E
:1043E00001D0FEF70DFE200010BD0124F9E7C04604
:1043F0008863FF1F70B500210600162005F0C8FF76
:104400000121152005F0C4FF07F01AFA0400092065
:1044100007F066FA00222B4B2B4DDA6661321A60E8
:1044200019685B3A9143002E28D0023A0A431A6079
:10443000AC4209D10A22DA6107321A6200221A63F9
:104440009A630132DA6370BD204A944203D11E227E
:10445000DA610532F1E71E4A944203D13022DA6173
:104460000632EAE71B4A944203D14322DA6108325A
:10447000E3E7194A9442E1D16922F7E702220A43AD
:104480001A604622AC4203D0104A944204D19422CE
:104490005A6106329A61D1E70D4A944201D1E6226F
:1044A000F6E70C4A944204D13422FF325A610D32AD
:1044B000F0E7094A9442C1D1E62252005A610A3219
:1044C000E8E7C046005000400024F4000048E8013E
:1044D000006CDC020090D00300D8B80510B50024B1
:1044E000064B0920DC6607F053FA2100162005F080
:1044F000E3FE2100152005F0DFFE10BD0050004056
:10450000F8B51C000023134D0F00EB666860160021
:1045100007F0AEF801238022EB6623002F615200E2
:10452000013B08D207F05CF808200B4A1168002C08
:1045300003D12000F8BD2A61F2E72B6F034203D0BC
:104540002B69013C3370013613685B1A032BEED9DB
:104550000124EEE7005000406008FF1F002370B503
:10456000124D1400EB6668600E0007F081F801231D
:104570008022EB6623005200013B08D207F030F89E
:1045800008200B4A1168002C03D1200070BD2A615D
:10459000F2E72B6F034203D02B69013C33700136E5
:1045A00013685B1A032BEED90124EEE7005000409C
:1045B0006008FF1F002370B50C4C0D00E3666060BF
:1045C00007F056F80123E366256107F009F880201B
:1045D000074A80001168636B034205D113685B1AB8
:1045E000032BF8D9012070BD0020FCE700500040EB
:1045F0006008FF1F002370B5134C0E00E366606077
:10460000150007F035F80123E36626610F33626B6E
:104610001A42FCD02B0A23611023626B1A42FCD091
:10462000EDB2256106F0DCFF8020084A80001168A9
:10463000636B034205D113685B1A032BF8D9012081
:1046400070BD0020FCE7C046005000406008FF1F1E
:10465000002370B5124D0C00EB666860160007F081
:1046600007F80123A619EB660F33B4420ED106F00A
:10467000B7FF80200B4A800011686B6B03420CD19E
:1046800013685B1A032BF8D9012070BD22782A61C8
:104690006A6B1A42FCD00134E7E70020F5E7C04618
:1046A000005000406008FF1F10B5084CE368002B65
:1046B00006D1074B1B680A336360064B1B682360F7
:1046C00007F016FA0002000AA06010BDB863FF1FD1
:1046D000C8F00040CCF0004010B50D4B986A9A6AC3
:1046E0008242FBD10B4A516894684118091B4B1E4A
:1046F000844200D30B0011689060D80B5B04401813
:104700005B0C10605360044A1360044B186010BDCA
:1047100000F00040B863FF1FC8F00040CCF000403C
:1047200010B51B4B1A793F2A01D93F221A7119790A
:10473000184A1948117018221849028018480A802E
:1047400002804A809A791748802402800C208A804F
:10475000013242432401101CA24200D9201C124AFB
:10476000C88010805A79002A01D101325A711A7A10
:10477000012A01D802221A725A791B7A0B48534334
:104780000A21584307F024F9094C206010BDC046A7
:10479000AC63FF1F480AFF1FFC43FF1FC845FF1FF4
:1047A000FA43FF1FA465FF1FF843FF1F71020000BB
:1047B000CC63FF1F10B508210020FEF709FE124C44
:1047C000002807D10C222000104907F0E1F9FFF77B
:1047D000A7FF10BD0C2220000D49FEF7CDFD0C28CF
:1047E00004D00C222000094907F0D2F9094C0C2210
:1047F00020000949FEF7C0FD0C28E8D00C2200215A
:10480000200007F0F5F8E2E7AC63FF1FBCBC001125
:10481000FC0C00008863FF1FF50C0000F0B50400DD
:1048200000200E00150085B082426ED0B7787278F5
:104830003F021743F2780B7812043A43377901317B
:104840003F061743039723706070262B00D179E051
:1048500010D8072B06D8180007F0E2F8513434348A
:10486000347D8B84232B00D1B4E0252B53D0FF2340
:1048700063708DE0712B00D182E01DD8562B46D09D
:10488000602B00D192E0552BF1D16A1E784D0C2A95
:104890003FD8002A09D0280007F07AF9FFF740FF37
:1048A0000C2228007349FEF7A1FC0C222900601C91
:1048B00007F06EF90D2028E0722B00D16AE0DC2BA6
:1048C00000D198E0DB2B00D0B0E0042DCFD9CB3B5A
:1048D0000193052D06D06B1F1A003800711D01933E
:1048E00007F056F905223100200007F051F9390090
:1048F000019A601D07F04CF90198053005E00C2283
:1049000020005D4907F044F90C2005B0F0BD5B497B
:10491000574D0C22BFE76A1E594D0C2A10D8002AA9
:1049200007D0280007F034F90C2228005549FEF77B
:104930005DFC13222900601C07F02AF91420E4E72B
:104940000C22EEE74E4D01001322280007F050F82C
:10495000FEF756FBEDE705224B49601C07F018F9FE
:104960000620D2E712224949601C07F011F91320F2
:10497000CBE708224649601C07F00AF90920C4E782
:104980007178F72900D972E7424B188801F00CFDC5
:104990000220BAE700F054FB012D03D03E4B7278A1
:1049A0005B6B1A6006F0D4FD0020AEE76A1E3B4D3B
:1049B000062A0DD8002A04D0280007F0E9F800F0F4
:1049C00079FF06222900601C07F0E2F807209CE727
:1049D0000622F1E7042D04D9314D2F6007F088F845
:1049E000A860FFF779FE0422039003A9601C07F07A
:1049F000CFF8052089E7022D00D838E77378BFB2D9
:104A00006370B378A370032D05D0033D3900AAB2BB
:104A1000F01CFEF7EBFB10223900E01CFEF7ACFCAB
:104A200003000330002B00DB6FE721E7DA2B00D017
:104A30001DE7042D00D81AE7082D16D9B37972792D
:104A40001B021343F27912041A43337A1B061343F1
:104A500003933B603B68052231002000039307F07D
:104A600097F80422601D03A986E7FE236370F1E72F
:104A7000AC63FF1FFC0C0000C8BC0011BCBC0011E3
:104A80008863FF1FF50C00009463FF1F7463FF1F12
:104A90003C45FF1FFE43FF1F00F000409944FF1FED
:104AA000B863FF1F70477047013870B5042809D8F4
:104AB00006F0B6FF0309250812001B4B02211878E7
:104AC00006F016FF70BD184B0821187806F078FF25
:104AD0000022164B1A72F5E70024144B124D0821E0
:104AE0001A6828781C8106F063FE2100287807F0F8
:104AF00037F8012000F016FE00F0DCFEE2E70A4B7A
:104B00000821187806F05CFF0948FFF7B9F9094B4E
:104B1000094A9B7900209380084A13808022034B26
:104B200052001A81E6E7C046C863FF1FCC63FF1F2F
:104B30000744FF1FAC63FF1FC845FF1FA465FF1F8D
:104B4000020010B5094B0A32094C92B2DA815A823E
:104B500098811882207802F08DFA0422054B0121F9
:104B600020781A7006F0C4FE10BDC046C644FF1F70
:104B70000666FF1F0566FF1F10B5012909D1054B09
:104B80001B78002B05D02622034B04485A72FFF7EE
:104B9000D7FF10BDD865FF1FCC63FF1FC4090000FD
:104BA0000300F0B50A4D8E18B14202D152008018B0
:104BB000F0BD0C782F6824093C5D0F271C700C7821
:104BC00001313C402F683C5D5C700233ECE7C0462D
:104BD000F443FF1F10B5114B1A781870002A0ED03D
:104BE00000280BD10E4B1A78062A07D85423D3403D
:104BF000DB0703D50B4B187802F03CFA10BD0028F8
:104C0000FCD0074B1B78012B02D0033B022BF5D8BD
:104C1000044B0121187806F06BFEEFE7D865FF1F03
:104C20000566FF1F0666FF1FF7B5624D624A6349BE
:104C30002870082005F072FC0121022005F06CFBB1
:104C4000022005F055FC0121002005F065FB002045
:104C500005F04EFC00F0ECFEFEF7D2F906F068FC21
:104C6000032257495748FFF79BFF2D2403000422D6
:104C70001C7055490130FFF793FF30230222047066
:104C800043708370514C524B2000DA8706F058FC79
:104C9000022815D0062220004E49FEF76DFB06289B
:104CA0000ED00321200006F063FD8D23E3706E3BE0
:104CB000237106221933200046496371FEF796FAE4
:104CC0000D23454F454C464E3B70013B04223000BE
:104CD00044492370033B6370019606F059FF2D236E
:104CE000012241494148A371FFF75AFF012240497F
:104CF000FFF756FF01223549FFF752FF0020FFF76B
:104D000069FF3C4E3C4A01213C4B1278307802F05E
:104D100073F9230000213A78307802F06DF901220E
:104D20002178374B01391A700020019AC9B205F079
:104D300069FD344B5A6B1268552A31D100225B6BE6
:104D400031481A60314B3C325A72FFF7F9FE20218C
:104D5000287806F0EDFE0120404205F09FFD01207D
:104D6000404205F03BFEFFF76BFAFFF76DF800F0ED
:104D70008DFC01204042FFF737F9012006F0D0FBFF
:104D8000F72001F0F5FA0121287806F0B1FD287826
:104D900002F0CCFA1E4806F07BFDFEF763FFF7BD7C
:104DA000FA210B4B1B4A49019981DA8119825A82F7
:104DB000CDE7C046C863FF1FA54A0011794B00111B
:104DC0003C45FF1F7463FF1F9463FF1F6509FF1FAE
:104DD000C644FF1FADAC0000D465FF1FB565FF1FC3
:104DE000B765FF1F7BBC00116709FF1FBC65FF1F74
:104DF0006609FF1F0666FF1F2644FF1F0744FF1FAB
:104E0000A665FF1F00F00040C4090000CC63FF1F2F
:104E1000D863FF1F4A1F0000F8B50A0020230D00C9
:104E20001A4019423ED0464B1B78002B37D0FFF773
:104E300053FC444C444E6368727AC31A934202D3C3
:104E40006060FEF70FFF327A217A531EDBB299427F
:104E500005D1FFF797FA002000F0D2FD0FE0914254
:104E6000F9D300232372FFF7B1FA012000F0C8FD47
:104E7000364F3800FFF704F8390006F019FE637A60
:104E8000002B09D0013BDBB26372002B04D1707997
:104E900064335843FFF754FE237A013323722020F2
:104EA0006840F8BD0BB2002B0ADA294B187806F0DF
:104EB000CFFB002801D006F053FB80200002EFE773
:104EC0000224214206D01F4B01201A72FFF782FEF6
:104ED0002000E5E70B0716D5FFF7FEFB194A1A4934
:104EE0005368497AC31A8B4202D35060FEF7BAFE68
:104EF000FFF76CFAFFF746FA012000F081FD00F0A1
:104F0000DFFB0820CCE71024214206D00C4B1B7895
:104F1000002BDDD1FEF7ACFFDAE70124214207D0F8
:104F20000C4800F065F806F05BFD00F0EBFCCFE705
:104F30000424080020402142B3D0FFF771F8C7E7EE
:104F4000D865FF1FCC63FF1FAC63FF1F0744FF1F23
:104F5000C863FF1FEC43FF1FF0B51B4B1B4F1B88A3
:104F60003A8804001A4E1B4D85B09A420DD83288FB
:104F70009A420AD3184B1A882B889A4205D1174AAD
:104F8000174B12881B889A421BD0052001F046FA65
:104F90003B8802AA13803388019053802B88114DDF
:104FA00093800F4B02A91B88D3800F4B2A78188857
:104FB00002F062FF0D4B08212878019A1C7006F060
:104FC00007FB05B0F0BDC046A265FF1FFC43FF1FF5
:104FD000FA43FF1FA465FF1FA065FF1F9E65FF1F0B
:104FE000F843FF1F0666FF1FFE43FF1F9C65FF1F60
:104FF00013B50C4B1C78002C11D1002801D00A4BA2
:1050000018600A4A0A4B11780A4A10780A4A019233
:105010000A4A0092002205F0EDFA200016BD112484
:10502000FBE7C0460566FF1F9865FF1F0466FF1F6C
:10503000F465FF1F0666FF1FE065FF1FE465FF1FA5
:1050400010B5064B12201B78052B06D1044B1322FA
:105050001988044B187801F0BDFB10BD0566FF1FD1
:10506000FE43FF1F0666FF1F10B500240122114BEF
:1050700052421870104B1C70104B1A8002F056F9F7
:1050800004220F4B21001A700E480C3206F0B0FCBF
:10509000102221000C4806F0ABFC07220B4B1C60D1
:1050A0000B4B1C700B4B1C700B4B1A700B4B1C707A
:1050B00010BDC0460666FF1F0566FF1FFE43FF1FAB
:1050C0000466FF1FF465FF1FE465FF1FE065FF1F17
:1050D000B465FF1FB365FF1F0044FF1FB265FF1FCC
:1050E000F8B5174C0600257806A814240078052D7D
:1050F00023D1B41F134FA5B21824BD421DD88D1F54
:10510000ADB2BD4219D8FA256D00AA4215D21D00D4
:105110000D4F0A3DADB2BD420FD80C4C26800C4C51
:1051200021800C4900240A800B4A1380FFF714FFEA
:105130000A4B0421187806F043FC2000F8BDC04655
:105140000566FF1F790C0000750C0000FC43FF1F73
:10515000FA43FF1FA465FF1FF843FF1F0666FF1FEA
:10516000F0B50BB20D0089B0002B00DB76E1A64E46
:10517000307806F06DFA041E55D00378A22B00D1CA
:1051800027E1D02B1AD0912B4AD143780E2B47D14F
:105190009E4B82889A4243D19D4A83681278052AA1
:1051A0003ED1032018567F283AD09A4B1B68002B1B
:1051B00036D05B68002B33D0984731E080780728E1
:1051C0002ED806F02DFC042D1D444479ADDD637806
:1051D000002B11D10622E11C8F4806F0D9FC0121D9
:1051E0008B4B19708D4B1A78002A5BD08C4B307822
:1051F00001F002FF002855D00722854B1A7051E0BC
:1052000061780029F8D1E378002B11D0854A864BCC
:105210001278307801F0F0FE60706378002BEBD1EB
:10522000200006F09DF980200002684009B0F0BD22
:10523000774B1B78022BF3D00121307806F0C8FAA7
:105240000028EAD10121307806F052FBE5E76378C7
:10525000002BD1D16E4F032807D13B78052B02D10B
:1052600001333B701EE00223FBE7704B1A88704B42
:105270000293002A0BD01B78002B03D00121307839
:1052800006F0A6F93B78062B04D1013BE9E7029B27
:105290001A70F7E7042B41D10121029B3078197075
:1052A00006F026FB5B4B1B68002BB9D01B68002B5C
:1052B000B6D0574A10787FE76378554F002B27D137
:1052C0000622211D5B4806F063FC62895A4B5B494C
:1052D0001A80A2895A4B1A80E3890B800521397004
:1052E00058490A80584A1380228A584B1A80584BD2
:1052F0001B78012B09D11F2001F090F8FA229200AF
:1053000042430421307806F063F90022484B75E7E8
:10531000312B00D070E70022454B1A700323A0E721
:1053200006220021434806F063FB0023454A04217E
:105330001380454A30781380444A138006F040FBBE
:105340000821307806F03CFBA379083B5A425341D0
:105350002F4A03331370314B1B78002B06D0344B8C
:1053600030781A78002A06D001F084FE0122324BF0
:1053700052421A8096E70121197006F0B9FAF5E752
:105380000821307806F01CFB6378002B00D047E73B
:105390002C4B2E4F0293E388029A042113802A4B50
:1053A000307803932389039A138063893B8006F046
:1053B0000FFA002800D033E7264B1B68002B00D1E2
:1053C0002EE7039902983A88098800881B68984755
:1053D00026E74379132B00D022E70389012B0AD15A
:1053E0001D4B1B78022B06D10821307806F0E8FA15
:1053F000FFF726FE14E7052001F010F8082102004F
:10540000307806F0E5F80BE70666FF1F051400008C
:105410000566FF1F9865FF1FD965FF1F2644FF1F04
:105420000744FF1FD465FF1FB565FF1FD665FF1F2B
:10543000D865FF1FA765FF1FFE43FF1FAE65FF1F57
:10544000B065FF1FA265FF1FA065FF1F9E65FF1FC0
:10545000A665FF1F9465FF1F9C65FF1F8020C0018C
:10546000014200D0E1E6CB0731D5324B1B78002B4F
:105470001DD0314E05AC3378052B1AD1023B237079
:105480002E4B21001B7823722D4B1B7863722D4B02
:10549000187801F055FD002809D007202A4B3070FC
:1054A0001B68002B03D01B68002B00D098470120FD
:1054B000BBE60E20254B06221B7825492370254B81
:1054C0001B78637002ABC01806F062FBD8E70223BA
:1054D00008001840194209D0174B1B78052B03D13F
:1054E0001D4B188806F0A4F802209EE604242142F1
:1054F00003D0FFF731FD200097E60823080018408D
:10550000194200D192E6154B1C78012C03D0022CD5
:105510000DD0082089E6124B124A134913481B8804
:105520001288098800880094FFF7DAFDF1E7FFF799
:1055300087FDEEE7D865FF1F0566FF1F0044FF1FCC
:10554000B265FF1F0666FF1F9865FF1FB465FF1F4A
:105550000144FF1FB365FF1FFE43FF1F9C65FF1F34
:10556000F843FF1FA465FF1FFA43FF1FFC43FF1F03
:1055700010B502A804880B20002C10D149680878C7
:105580004978090201430C48814209D1022119805E
:105590000A4B59881170DB7800205BB2537010BD44
:1055A000074C0A20A142FAD102211980034B9988A5
:1055B00011705B79F0E7C0466E2A0000A063FF1F00
:1055C0006F2A0000F7B5150008AA16884A680F4F21
:1055D00014785278120222430A24BA4214D10122CA
:1055E000DBB2019200962A0005F00AFF041E0BD1DF
:1055F000074B1B68002B07D068782A7800021043FD
:1056000042425041013098472000FEBD022900006F
:105610001866FF1F30B5012503790400BFB02B4287
:1056200027D01549408805F057FA28420DD06A4620
:10563000124B69465B8D138002235380104B5B88AD
:1056400093806088002202F00DFB0E49608805F00F
:1056500043FAC0070DD56A460B4B69461B88138079
:1056600002235380064B9B8893806088002202F0BF
:10567000F9FA3FB030BDC0461066FF1F2844FF1F37
:10568000A063FF1F0866FF1F8244FF1F10B5074C71
:105690000749200005F0D6F92000064905F0D2F9A7
:1056A0000721054A054805F08FF910BDFFFF0000EE
:1056B0001066FF1F0866FF1F48BD00112844FF1F2A
:1056C00010B5024803F050F910BDC0461556001140
:1056D00070B55F25082607498400CA788B78400199
:1056E0002A40B3433440A843234302438B70CA701B
:1056F00070BDC0469944FF1F010043B204205A0008
:1057000002409B000C3003401A43152310B5044C93
:10571000E0789843143B0B4018430243E27010BDFD
:105720009944FF1F10B5054B082419790A00A243BC
:10573000002801D022000A431A7110BD9944FF1FAE
:1057400010B5054B4024D9780A00A243002801D0A7
:1057500022000A43DA7010BD9944FF1F0821F8B5F2
:10576000324D334BAE7804000E40AE70984204DDEB
:1057700067232B70473B6B70F8BD2E4B984203DAC2
:10578000E0232B703A3BF6E700232B706B7083B25B
:105790001A0029485F3292B2284F82422CD9002C3D
:1057A00003DA5B421CB204232B70053420B20A21B9
:1057B00006F00EF904B2FA239B009C4232DB082368
:1057C0002A7813432B706421200006F001F90A2186
:1057D00000B205F0DDFF09B22A787B5C13432B7021
:1057E0000A21200006F0F4F80A2100B205F0D0FFEB
:1057F00009B27B5C6A780AE06970002CDBDA5B42F4
:105800001CB204232B70F3226B78092CE8DC1343C1
:105810006B700A21200005F0BBFF09B27B5C1E43C0
:10582000AE70A9E7632CCEDCEDE7C0469944FF1FBC
:105830001B4E00001DFCFFFF2A0800006FBD001179
:105840000823F7B5194FCD003E7904001E403E7184
:10585000EDB2632806DD5F3333433B7120231D43E4
:105860007D71F7BD0300093305DA20235B42334322
:105870003B71A623F3E70E4B019300280BDA0423B8
:10588000444224B23B710A21200005F081FF019BB4
:1058900009B25B5CE3E70928F5DD0A2106F098F818
:1058A000019B00B21B5C1E433E71ECE79944FF1F55
:1058B0006FBD001170B50F4B1B78002B18D00E4E2A
:1058C0000E4D06223100280006F0C2F800280FD045
:1058D000062231000A4C280006F0E2F80120FEF70B
:1058E00089FD072221003E20FEF7B2FEFEF7F6FDFD
:1058F00070BDC0462466FF1F9944FF1F1E66FF1F30
:105900001D66FF1F10B50820FFF728FFA622024BD7
:105910001A70FFF7CFFF10BD9944FF1FF8B51C4B5D
:105920003C21186806F03CF83C21040006F080F8A1
:1059300020000F003C2106F033F8182106F078F81B
:1059400000230E00134C0A212370300006F028F8C3
:10595000114D0A212B5C3000637006F069F840227B
:105960006B5C2679A370E37838001340E37008235A
:105970000A211E4006F014F82B5C0A211E43380051
:10598000267106F055F86B5C6371FFF793FFF8BD65
:10599000B863FF1F9944FF1F6FBD001110B5164C6F
:1059A0000A210223E05E06F013F800B2FFF7D6FEEC
:1059B0000423E05E642106F00BF8012100B2FFF73A
:1059C0003FFF237A0024132220009A426041C0B294
:1059D000FFF7B6FE0320FFF77BFE2000FFF78CFEEB
:1059E000064B1878053843425841C0B2FFF79AFE7B
:1059F000FFF760FF10BDC046A063FF1F0566FF1FD5
:105A0000094B10B51A6801231A4208D007490A78D1
:105A1000D01808701A4204D0FFF780FF10BD00288C
:105A2000FCD0FFF7BBFFF9E7AC63FF1F1C66FF1F4D
:105A3000002010B5FEF7DEFC0D223E200549FEF7E2
:105A400007FE0023984200D13E33034A1370FEF74D
:105A500045FD10BD62BD00112466FF1F0200F0B5B8
:105A600001270A480A4E51188B1A002B00DCF0BDA2
:105A7000082415784308684038404000805B013CAA
:105A800058406D08002CF5D10132EDE7FFFF000012
:105A900080BD0011F0B500250F269D4200DBF0BD52
:105AA0004C5D070944403440A400A05801357840BB
:105AB000F3E70000F0B589B06A460D000B000F2730
:105AC000110010351C780133260024093E40167061
:105AD00054700232AB42F5D12023024AFFF7DAFFBD
:105AE00009B0F0BD84BD0011F0B54E780B7889B0D7
:105AF00036020C00170001901E43012A61D9974B12
:105B00009E4200D878E001339E421CD1062A17D16C
:105B1000CA788B7812021A430B791B0413434A7913
:105B200012061A438E4B5A6100221A705A808D4A0F
:105B30005A608D4A9A608D4ADA60002009B0F0BD43
:105B400088225205EEE78A4B9E423CD184498B78ED
:105B5000002B00D0FAE00C2A31D10F22A378934316
:105B6000E278120213432279120413436279120677
:105B700013434B60E279A07912020243207A0004B9
:105B80001043627A12060243CA60E27AA07A1202D5
:105B9000024378484A81834208D80423704914227A
:105BA00001980B7005F0F4FF1420C7E71201D2181A
:105BB00089235B059A42F0D801238B70BDE7022A46
:105BC000FAD00523EAE76C4A01239642E6D1FFF7B3
:105BD00037FA052F0DD9E378A2781B0213432279F7
:105BE00012041A4363791B061343644A0393526BEE
:105BF000136005F0ADFCA0E7594D2B78002B9CD12C
:105C0000AB78002B00D1A3E02B8901339BB200932A
:105C1000B34200D094E0132AD3D9CF7C8B7C3F02CF
:105C2000122120001F43FFF719FF874200D091E0A7
:105C3000002E3ED1E378A2781B0213432279E96853
:105C400012041A4363791B06134303930A228B42FF
:105C500013D1FF23A370E370237163716B89002B51
:105C60000AD1E37B227C1B0212041343A27B134361
:105C700003931B0901336B8100226B89002B8CD0AD
:105C8000002A69D1686837013818000B6B69000376
:105C90000390984205D9686105F06AFFEB780133FB
:105CA000EB7068681022A11C381805F049FD2E81A0
:105CB00043E76F89009A7B1E9BB293423CD1E37805
:105CC000A2781B02134322792D4E12041A436379E2
:105CD0006C681B0613433100042204A8039305F0EB
:105CE00057FF211D0C2205A805F052FF012004A931
:105CF00040421034FFF7DEFE013F012F17D1039A17
:105D00000B232861824200D048E7042231006868F2
:105D100005F016FD042203A9686805F029FEE9686C
:105D2000039AFF23914200D138E7F73B36E7210081
:105D3000FFF7C0FE1034DFE70923B742A2D82DE7F2
:105D4000009BB34200D9F8E6072327E7022325E7A3
:105D5000032323E7062321E70A231FE7FFFE0000B2
:105D6000A044FF1F00000111FFFF000050485936FA
:105D700001FF0000FFFF001102FF000000F00040E3
:105D8000AC44FF1F10B5034C0B000122210000F0B2
:105D90006BFA10BD455F00110B8870B506000D0051
:105DA0000224162B11D92B000322094900F05CFABA
:105DB000041E0AD1074B2A881B88191C934200D95C
:105DC000111C300089B200F0EFFA200070BDC0460F
:105DD000715F00117E66FF1F10B54A780400013A1A
:105DE0000B000220012A07D80A78002A04D00522D5
:105DF0002000024900F038FA10BDC0469F5F001134
:105E00000A7810B50B0004000220002A04D00722F3
:105E10002000024900F028FA10BDC0464B60001176
:105E20000A7810B50B0004000220002A04D00922D1
:105E30002000024900F018FA10BDC046B160001100
:105E400010B5034C0B000B22210000F00DFA10BD21
:105E5000E160001110B5034C0B000D22210000F091
:105E600003FA10BD5361001110B5034C0B000F2253
:105E7000210000F0F9F910BDAD6100110A7810B5EC
:105E80000B0004000220002A04D011222000024945
:105E900000F0EAF910BDC046BD610011002310B545
:105EA0001322190000F0E0F910BD000010B5034CFA
:105EB0000B001722210000F0D7F910BD0F6200116E
:105EC000002310B51922190000F0CEF910BD000012
:105ED00010B5034C0B001B22210000F0C5F910BDCA
:105EE00049620011F7B584890D0006000121002CDC
:105EF00022D000238268D3561778002B1EDA0C2C90
:105F00001AD90C3CA4B2131940880093230002F064
:105F100086FE431E984101307B06DB0F6B703F23EA
:105F2000013C1F40A4B22870AF70AC80002C07D099
:105F3000B3680133AB6000210800FEBD0020EBE731
:105F4000AC60F8E70B7803704B8843704B881B0AF2
:105F500083700B79C370042070470420022B06D194
:105F60000020537811781B02009A0B43138070476E
:105F70000B8803700B881B0A4370022070470420B3
:105F8000009983420AD1537810781B0203430B8097
:105F9000D37890781B02034300204B807047F8B5FC
:105FA0000D004B7801240021461C03702B788B4296
:105FB00001D82000F8BD6B78B01C4F1C012B10D10C
:105FC000890069184B88022233704B88B9001B0A7C
:105FD0007370691805F0DCFD04360434A4B2F9B21C
:105FE000E4E7122359436B185A88043132705B88F6
:105FF00010221B0A7370691805F0CAFD123612349C
:10600000ECE770B5049D14001E00052B01D8042098
:1060100070BD637812781B0213432B80E378A2785B
:106020001B02134302226B802A71211D681D063E4C
:1060300005F0AEFDB2B22A81F02AE8D82800A11DF1
:106040000A3005F0A5FD0020E2E7002310B50A782C
:106050009A4201D8900010BD9A008A1854880133E2
:1060600004705488DBB2240A447094888470928847
:10607000120AC2700430EAE710B51100029C062B28
:1060800004D004201022142B01D010BD0222227152
:106090004B7808781B0203432380CB7888781B0257
:1060A000034363800431601D05F072FD0020ECE7BE
:1060B00010B50C788B7804315C43E4B20370220095
:1060C000013005F065FD601C10BD0420022B06D1D7
:1060D0000020537811781B02009A0B4313807047FD
:1060E00010B50C000A88023105F052FD208810BD61
:1060F00070B504000D0004981100012B01D8042094
:1061000070BD167852781202324302800200F832D3
:1061100055701470E825002C00D10C35023B9AB262
:106120004280AA42EBD80231043005F031FD002054
:10613000E6E70420009983420AD1537810781B02C5
:1061400003430B80D37890781B02034300204B80DD
:10615000704710B50C000A88023105F019FD20883F
:1061600010BD000070B501211E000420049C0E40EB
:106170000B4218D1CB40DDB28D4214D90A49DBB2B3
:10618000098899420FD32300F6331D70330058005D
:1061900011184978165C0902314301332152D9B2F2
:1061A0008D42F4D8002070BDC044FF1F10B50C0014
:1061B0000A88023105F0ECFC208810BD10B50C787F
:1061C0008B7804315C43E4B203702200013005F0A7
:1061D000DFFC601C10BD10B511000298032B01D824
:1061E000042010BD14785278043B1202224302802E
:1061F000CA788C781202224342809AB28280F22AB4
:10620000EED80431063005F0C3FC0020E9E710B5F4
:106210000C000B8803700B881B0A43704B8883703B
:106220004B881B0AC3708A880430063105F0B0FC25
:10623000A088043080B210BD0420012B03D10020BF
:106240001378009A1370704710B50C000B88037018
:106250000B881B0A43704A880230043105F098FC11
:106260006088023080B210BDF0B589B003931E4B38
:10627000029242000700D05A019102F020F8132543
:10628000061E2DD0029B01240370019B002B04D01D
:10629000001903999847001984B26B461B7A5BB2C8
:1062A000002B0FDA1021380002F01CFB1925002802
:1062B00013D130003219E1B202F066FC051E0CD198
:1062C0000C34A4B2042304AA380005A993800696CE
:1062D000948101F0AFFD051E02D0300005F090FA68
:1062E000280009B0F0BDC0467C66FF1F70B50500F0
:1062F0000C0000280CD00020814209D01022200080
:10630000044905F045FC01202B7823736B786373F7
:1063100070BDC046C4BD0011F0B506000D001700E9
:106320001C0085B002291BD00020102907D1022BA8
:1063300007D0102B03D115E00020102C08D005B099
:10634000F0BD69463800FFF7D1FF2A0069460BE02F
:1063500069463000FFF7CAFF22006946380004E0B2
:10636000022BE9D12A003900300005F081FBE6E775
:10637000031CF72800D9F723032008499AB2013AF1
:106380000B80D317034006499B189B100B80D30F3B
:1063900004499B185B100B807047C046C444FF1F24
:1063A000C244FF1FC044FF1F034B1B888B4202D314
:1063B000024B4000C1527047C444FF1F7C66FF1F60
:1063C000014B4000185A70477C66FF1F1722014B93
:1063D0001A8070477C66FF1F70B505000E2005F01F
:1063E00097FA041E13D0D023037000230622837073
:1063F00007494570033005F0CBFB064B2100DA8AD4
:1064000062811B7E2373044B187805F069FB70BD15
:106410009866FF1F8866FF1F1445FF1F262803D8B4
:10642000024B4000C05A70470148FCE7C644FF1FBA
:10643000FFFF000070B506000C00094D1C22002172
:10644000280005F0D5FA074B1E70074B1C7005F0AD
:1064500097FB0123002801D0002312202B7070BD70
:106460008866FF1F1445FF1FA966FF1F70B5050052
:106470000D4C0800E260A16010220021656005F06B
:10648000FFF9012803D11021A06802F058FD102265
:106490000021280005F0F4F9012803D110216068DB
:1064A00002F04DFD70BDC0468866FF1F70B5041E2A
:1064B00005D1002903D006220D4805F069FB0D4BDC
:1064C0001D78012D11D1002C05D102221A7005F082
:1064D000FFFA280070BD00221A70074B1B78FF2BB3
:1064E000F7D02000FFF778FFF3E70025F1E7C0467B
:1064F0009866FF1F8866FF1F1445FF1F030010B535
:10650000002801D1002010BD00780B4A002803D1DB
:106510005988D1821B7913761378022BF2D100238C
:10652000984200D103331370044B1B78FF2B01D02A
:10653000FFF752FF0120E6E78866FF1F1445FF1FA3
:10654000002911D000280CD04B79012803D140221A
:106550005242134303E03F221340032802D001209C
:106560004B7170474022F4E70800FAE770B5094D17
:106570000100287800280BD0074C0622200005F0E7
:1065800007FB21002878FFF7DBFF200005F0F8F972
:1065900070BDC046A866FF1F8266FF1F00290AD093
:1065A000012808D13F224B799343C02B03D0403BB5
:1065B0005A425341981C704770B5174D06002B780E
:1065C000FF2B15D00A2005F0A3F9041E10D0D0230C
:1065D0000370C83B8370114B11491B784670C37020
:1065E0000622043005F0D4FA2100287805F078FA64
:1065F0000C4B1B78012B0DD10B4B1B68002B03D0D0
:106600009B68002B00D09847084B04211878084A53
:1066100005F0CEF870BDC0461445FF1FA866FF1FE9
:106620008266FF1FA466FF1FD066FF1FD466FF1F90
:1066300060EA0000014B98687047C0468866FF1FFB
:10664000014BDB68186870478866FF1F074B10B561
:10665000DA68136801331360054B1878FF2803D0FC
:106660008021C90105F044F910BDC0468866FF1FAE
:106670001445FF1FF7B50E0002F0C8F8051E1CD028
:106680000E4B06621F78002F00D10778AB791020DF
:10669000019305F03DF9041E0FD0D0230380C73BC2
:1066A0008370019BE91DC3700622043005F070FA67
:1066B00021003800E66005F013FAF7BD1245FF1F10
:1066C000014B18787047C046A866FF1F054B00288D
:1066D00005D1054B1A78054B002A00D1014B180053
:1066E0007047C0469866FF1FA866FF1F8266FF1F9F
:1066F000014B58687047C0468866FF1F024B1868F8
:10670000431E9841C0B27047AC66FF1F421E030093
:106710000120152A03D9FF3B5A425341D8B2704792
:10672000F0B51C0000230E0085B0039002920B70A0
:10673000029A934201D3002019E0E55C5A1CD2B2C0
:10674000002DF8D0029851198142F4DC0233DFB2F7
:10675000A35C18000193FFF7D9FF002807D0013D83
:10676000019A0399EBB233708A4202D1E01905B065
:10677000F0BDDB19DBB2DBE710B50C0002F09EF8D0
:1067800003001220002B03D02100588805F008FADE
:1067900010BD000070B50E4D84006359002B15D05C
:1067A000186A002801D005F05BF82B59586A0028B8
:1067B00001D005F055F82B59986A002801D005F052
:1067C0004FF8285905F04CF800232B5170BDC046F6
:1067D000B866FF1F1C4B70B504000E0015009942EF
:1067E0000AD11A4B1B68002B01D1122070BD1B6807
:1067F000002BFAD09847F9E7154B994215D1134B66
:106800001B68002B0AD01B68002B07D09847002874
:1068100004D1104B1C70104B1D70E7E729002000BD
:10682000FFF7AAFF0028E1D1F3E7080001F0EEFF2F
:106830000028DAD003780320A342D7D12900300002
:1068400005F0AEF9D2E7C046FEFF0000B466FF1FB8
:10685000FFFF0000B166FF1FB066FF1FF7B5040021
:10686000808801F0D3FF0025A84203D00578A088D6
:1068700002F008F81C4E3378002B1FD0AB421DD11C
:106880001A4B28001978FFF777FF002818D000234B
:106890003370A3790820A778A688019305F038F80B
:1068A000011E0DD0D0230370CA3B8370019B47703B
:1068B00086808371280005F013F901E0002DE8D1EE
:1068C000A0880B4B8200D358002B01D0FFF762FF4A
:1068D0001721A088FFF768FDA08801F027FDA08898
:1068E00001F0FEFDF7BDC046B166FF1FB066FF1F99
:1068F000B866FF1FF0B587B01D000CAB1B88070002
:1069000001930DAB1B88142002930EAB1B8816005D
:1069100003930FAB1B880091049310AB1B88059366
:1069200004F0F6FF041E1AD0D0230370CB3B47704F
:106930008370C670062229000430002D11D005F0A6
:1069400027F9019B21006381029B0098A381039B8F
:10695000E381049B2382059BA37405F0C1F807B073
:10696000F0BD05F045F8ECE7F7B5009308AB1B88E0
:1069700007000C200D001600019304F0C9FF041E4F
:1069800013D0280001F042FF00280FD00078D02358
:106990002370C93BA370009B21002381019B67707A
:1069A000A580E680638105F09BF8F7BD014B187860
:1069B000EDE7C0461445FF1F13B504006489038941
:1069C000C2888188C0780094FFF7CEFF13BD000015
:1069D00010B5044C2068002803D004F041FF0023C8
:1069E000236010BDBC66FF1FA122F0B58188920014
:1069F0004A43384B384F1B6804009B189D22920075
:106A00009B18827989B01A603B68002B5FD01D7893
:106A1000324B1B68002B04D05B68002B01D0002098
:106A20009847260008363100E079FFF7B7FD237D4F
:106A3000E0710200E0780493638A29000393238ABB
:106A40000293E3890193A38800933300FFF752FF79
:106A5000E378002B0BD1E289A379A18802920196F9
:106A6000E27928000092012201F0DAFEE0703B6832
:106A7000002B20D0FFF7ACFF194D287800281AD042
:106A8000184B1978FFF778FE002814D02B78E67899
:106A900008200793A78804F03BFF011E09D0D023EC
:106AA0000370CA3B4670837087808671079805F033
:106AB00017F800232B701721A088FFF775FCA0881A
:106AC00001F034FCA08801F00BFD09B0F0BD064BCD
:106AD0009DE7C0463409FF1FBC66FF1FD066FF1F3D
:106AE000B166FF1FB066FF1F1445FF1FF8B5070012
:106AF00008000E0001F08AFE041E18D02620FFF7C1
:106B00008DFC051E00D12578062004F001FF041E2F
:106B10000DD00021062204F06BFFD0232370C23B6E
:106B200021006770A370A680E8B204F0D9FFF8BD19
:106B3000F0B585B001930AAB1B78070002930BAB4D
:106B40001B7808000D000092039301F05FFE061E03
:106B500022D0102004F0DCFE041E1DD010220021E3
:106B600004F046FF2620FFF759FC002800D13078BA
:106B7000D0232370C13BA370009B21002372019B93
:106B800067706372029BA580A372039BC0B2E3721D
:106B90000C9BE36004F0A4FF05B0F0BDF7B50D0059
:106BA000019001F033FE071E20D00E2004F0B0FE4D
:106BB000041E1BD02620FFF731FC061E00D13E78B4
:106BC000D0232380C53B0622A370F91DE01C04F0EE
:106BD000DFFF019B2A0063810123DD401A401D4035
:106BE000210022736573F0B204F07AFFF7BD000054
:106BF000F0B585B0029010000D0017000A9E0393B7
:106C000001F004FE041E31D0029B002B2ED1039B09
:106C100002795B0724D5122313430422002E08D1E6
:106C20000B99002905D10C99002902D10D99002951
:106C30001AD01A430D9B2271002B00D0C9E0002E00
:106C400000D1CFE0002D00D0CCE0606A002801D058
:106C500004F006FE1C21300004F01AFD606205E01D
:106C600002239A430E33D7E793432371654BBA004F
:106C7000D458002C00D1AAE0002E10D0236A002B9B
:106C800003D11C2004F024FD20625E4BBA00D358CF
:106C9000186A002803D01C22310004F079FF0C9BF5
:106CA000002B12D0574CBB001D596B6A002B03D12F
:106CB000162004F00DFD6862BB00E358586A0028F6
:106CC00003D016220C9904F063FF0D9B002B11D00A
:106CD0004C4DBC006659B36A002B03D1142004F05C
:106CE000F7FCB0622B59986A002803D014220D9942
:106CF00004F04EFF380001F089FD051E67D0414BBE
:106D0000BA00D358002B62D01A6A3420002A00D16E
:106D10001C389A6A002A01D0143080B20B9A002ADB
:106D200001D01C3080B25B6A002B01D0163080B2DB
:106D300004F0EEFD041E4AD01822002104F058FE93
:106D40002620FFF76BFB0190002801D12B780193DF
:106D5000D0232370029B200063700A23294EA37066
:106D6000039BBD00A371AB59A780196A1830002995
:106D700005D01C22A06004F00BFF200034307359B2
:106D8000996A002907D0030014221433E0600293AB
:106D900004F0FEFE02980B9B002B08D003001C227F
:106DA0001C330B992061029304F0F2FE0298735990
:106DB000596A002903D01622606104F0E9FE6B468F
:106DC0002100187904F08CFE3800FFF7E3FC05B0D1
:106DD000F0BD10220D9B0D991B69A018236204F0D1
:106DE000D7FE2CE70B9B002B00D13FE7012D00D0F5
:106DF0003CE7606A002801D004F032FD1C210B98AA
:106E00002AE7C046B866FF1F10B5044C206800286A
:106E100003D004F025FD0023236010BDAC66FF1FE6
:106E20000B4B07B51A68002A01D100200EBD694638
:106E3000531C012012780731FFF772FC0028F4D0B0
:106E400002780123100018401A42EED0EEE7C04647
:106E5000C866FF1FF0B51F4F01203B6887B0002BAD
:106E600025D09B78059300F0B3FB002821D00A20A1
:106E7000FFF7D4FA04000B20FFF7D0FA164B0500F9
:106E80001E78731E9E413B68F6B2191DD878FFF735
:106E900057FB3B682900DA7A043303929A7901930D
:106EA0000292009033002000059A04F0F9FC07B02C
:106EB000F0BDFFF7B5FF002805D00620FFF7AEFABA
:106EC00004000720D8E70820FFF7A8FA04000920EB
:106ED000D2E7C046AC66FF1FA866FF1F70B50A4E1A
:106EE000040033780D00FF2B0DD0042004F010FDBA
:106EF000011E08D0D0230370CE3B45708370C47050
:106F0000307804F0EDFD70BD2445FF1F70B504001E
:106F100006200D0004F0FCFC011E0AD0D0230370F3
:106F2000CD3B8370054B44701B688580187804F056
:106F3000D7FD002C01D0FFF767FF70BDAC66FF1FC7
:106F4000F8B5264F06003B680D001124002B05D133
:106F50000522234B1B78134202D112242000F8BDD6
:106F6000204A10241268002AF8D01278002AF5D09E
:106F7000DB0719D52B789A1E012A1AD80C2004F0A9
:106F8000A7FB132438600028E8D000230A224370AE
:106F900029000670023004F0FBFDFFF75BFF041EC2
:106FA0000AD0FFF731FFD9E700F012FB0028E1D14A
:106FB000E4E7002BE2D0D0E70B4B1B78032BCDD1BD
:106FC0001D20FFF72BFA094B18800028C6D0084B6C
:106FD00004211878074A04F0EBFBBFE7AC66FF1FFB
:106FE000A966FF1FC866FF1FA866FF1FA666FF1FD2
:106FF000D466FF1F60EA0000F7B50193194B140037
:107000001A78052306000F0012201A4221D0012908
:1070100020D1154B1D68002D1BD002201F2C18D825
:10702000002C02D0019B002B13D0104B1F221E708E
:107030006E1C0021300004F0DBFC019922003000BE
:1070400004F0A6FD310020002C70002F06D004F0C3
:10705000DFFBFEBD064B12201D68DCE704F010FDCF
:10706000F7E7C046A966FF1FC866FF1F2445FF1F3C
:10707000C466FF1FF8B50F4E12243368002B17D0DB
:107080001B780F3C834213D100250B4F0221387827
:1070900004F096FC094B042138781D8004F090FC24
:1070A000074B28001D8033685C7004F001FC04006D
:1070B0002000F8BDAC66FF1FD466FF1FC066FF1F2F
:1070C000A666FF1F70B5012823D11B4C2388002B17
:1070D00003D01A4A1578002D07D0194B1B68002BD6
:1070E00002D01878FFF7C6FF70BD3B2B02D93C3B9E
:1070F0002380F9E7134E0221307804F061FCFA2274
:107100002388920002215A43307804F061FA2580E6
:10711000EAE70B4B1B68002BE6D00B4B1B785B0799
:10712000E2D5084B0221187804F04AFC0022024BF9
:107130001A80FFF769FED7E7C066FF1FA466FF1F2E
:10714000AC66FF1FD466FF1FA966FF1FF8B51E4D72
:107150002868002803D004F083FB00232B601B4E1B
:107160003068002803D004F07BFB00233360184F05
:1071700005243B7818002040234221D0154800F018
:107180002BFA3B78234213D0202004F0A1FA286088
:10719000002813D02022002104F02AFC202004F033
:1071A00097FA041E306005D02022002104F020FC54
:1071B000002004E0286804F053FB2C601320F8BD85
:1071C00000F00AFAF4E7C046C866FF1FC466FF1F56
:1071D000A966FF1F1845FF1F10B50A4C23681A1E29
:1071E0000ED0002808D10130587004F061FB00284F
:1071F00005D02368002B02D00021FFF787FE012273
:10720000100010BDAC66FF1FF7B5274E05003368B0
:107210000191181E21D05C78244F012C30D1FFF74A
:10722000FFFD002825D02000FFF7F8F804004128D2
:1072300014D91F4B022118781E4A04F0B9FA1E4BCC
:107240003C3C1C80022233685A703B78002B14D1DE
:1072500028000199FFF75AFE0120FEBDFA22920094
:107260004243002AEED0124B0221187804F0B0F904
:10727000E8E7FFF7D3F80200F3E700233B70EBE702
:107280003B78002BE8D1032004F042FB011E08D01C
:10729000D0230370CC3B457083703368187804F0BA
:1072A0001FFCFFF7B1FDD7E7AC66FF1FA466FF1F09
:1072B000D466FF1F60EA0000C066FF1F10B51749C3
:1072C000838802008B4220D011D815498B4217D0F9
:1072D000144900205B1899B2012907D892681178E7
:1072E0005A425341D8B2FFF7F9FD012010BD0E4AB2
:1072F00000209B1807229BB29A424041C0B2F5E79A
:1073000083681878FFF768FFF0E7836899785A7800
:10731000090218781143FFF777FFE7E70A2000001A
:1073200006200000F8DFFFFFAFDFFFFF014B187002
:107330007047C0462545FF1F10B5064C207001F070
:1073400041FA207804F02CFA0521207800F062FD43
:1073500010BDC046D466FF1F0BB273B50D00002BE5
:1073600000DBC4E0884B187804F072F9041E0ED0DC
:107370000378912B0FD0A22B00D1A1E0834B18787A
:10738000FF2852D0210004F0ABFB00284DD1802013
:107390000002684076BD43780F2B76D013D8052BBA
:1073A00070D00E2BEAD18088794B98422BD8794B3C
:1073B00098421BD8784B9842E0D1A3681878591CA2
:1073C000FFF774F838E03E2BD8D18378032B74D0C4
:1073D0006CD8012B6ED0022BD0D1704B1B68002BC8
:1073E00023D05B68002B20D098471EE06C4BC01860
:1073F0000C28C3D804F0E4F91DC2C2150BC20B0B54
:107400000B3223C23C00674BC0180728B6D8664B26
:107410001B68002B09D01B68002B06D02000984762
:107420000AE0A3681878FFF7C7F8200004F098F87E
:10743000ADE7A068FFF762F800289FD0F5E7A368E2
:107440001B78002BF1D0554B1B68002BEDD01B682F
:10745000002BEAD0210055489847EDE74F4B1B68B9
:10746000002BE2D01B68002BDFD021005048F3E74F
:10747000504B1B68002BD8D05B68002BD5D0210067
:107480004348E9E7FFF7EAF9CFE780884A4B98429B
:1074900003D04A4B984200D070E7464B1B68002B44
:1074A000C3D05B68002BC0D02100D5E7153B012B72
:1074B000BBD963E7FFF798FAB7E7FFF77DFAB4E7C0
:1074C0003F4B1B78042B07D100236A4613800179B8
:1074D000408800F0C5FCA8E7364B1B68002BA4D001
:1074E0005B68002BA1D00100364898479DE7012436
:1074F00021420AD0294B1B68002B04D05B68002B6B
:1075000001D000209847012043E78B070AD5264B7E
:107510001B68002B04D05B68002B01D0200098472B
:10752000022036E70421280008400D4200D131E74F
:10753000254E3388002B21D0013B9BB23380002B9A
:107540001AD1FFF7DBF800280AD0204B1C70164B2D
:107550001B68002B04D05B68002B01D020009847EB
:10756000FFF7C6F8694601F001FD6846FEF7FEFF29
:107570001D20FEF753FF308004200AE7024B1878E5
:1075800004F01EFAF8E7C046D466FF1F2545FF1F2A
:107590000E2000000120000009100000CC66FF1F33
:1075A000FEDFFFFFAFDFFFFFD066FF1F0C200000F4
:1075B0000B200000B466FF1F0D2000001320000008
:1075C000A966FF1FFFFF0000A666FF1FA466FF1F3E
:1075D00010B501F09BF910BD014B18607047C04613
:1075E000D066FF1F0B880020162B01D8172304201C
:1075F000014A13807047C0467E66FF1F0020704717
:10760000074A03001188814207D0918800209942DF
:1076100002D101308000101870470020FAE7C04600
:10762000DC66FF1FF0B58F7806000D00C7B01E2F77
:1076300015D1FFF7E5FF051E03D10024200047B058
:10764000F0BD00223B003100C078009200F0B2FB98
:107650000400A81C00F0D3FBFF23EB70EEE7264BE1
:10766000062403931B78FF2BE8D0182FE6D87B085D
:10767000224A013BDB0002929A589446002ADDD050
:10768000029AD3185B68002BD8D00878002802D162
:107690004B78012B02D10624122FCFD107AFAB8834
:1076A000697800976446AA68A047041EC6D1AB78E3
:1076B000029A5B08013BDB00D318390030005B689D
:1076C0009847041E0BD1AB78042BB6D0039A310037
:1076D00010782200009700F06DFB0400AEE76A7896
:1076E000002AABD1AA7805A93B88087130000A703E
:1076F0004B80FEF747FBA0E72845FF1FD4BD0011D4
:107700001D4B37B5050098420BD000290AD1FFF771
:1077100077FF002805D11948FFF772FF002800D035
:10772000058037BD01291AD1FFF76AFF041EF8D082
:1077300001235B420380A378FF2BF2D0FE2B07D0FE
:107740000023E0781422009329001E3300F032FB5E
:10775000A01C00F054FB01235B426380E1E7022997
:10776000DFD1013901F0BEF80028DAD12800FFF797
:1077700047FF041EDFD1D4E7FEFF0000FFFF00003B
:10778000022210B5074B52421A80074801325A8034
:107790009A80DA8000F07EFA044801F025F8002093
:1077A00010BDC046DC66FF1F257600110177001171
:1077B0000388F7B50400002B02D102252800FEBD86
:1077C00042680221137825485268FEF7A5FD00287B
:1077D0002ED0234F01253A88002AEFD0802321881C
:1077E0005B0201259B1A9942E8DC0C2003F070FF34
:1077F000061E31D03B8822889C4600231800019544
:1078000061469DB2491989B2AA421BD8002801D00D
:1078100062443A8000233000082208C0210004F0AE
:10782000B7F9104A1368002B13D100251660C5E77D
:107830006268022113780C485268FEF76DFD00283B
:10784000C7D1BAE760681D01401941810133019831
:10785000D6E71A001B68E6E71325AFE742BE001122
:107860002645FF1FD866FF1F40BE0011014B187050
:107870007047C0462845FF1F14230A0010B51A4060
:10788000194204D00122102101F048F810BD4B0626
:10789000F9D4012088434000F8E710B514008B06A6
:1078A00004D50122102101F039F810BD08230A0087
:1078B0001A40194202D14BB2002B0FDA102101F00D
:1078C0002DF8002808D02300F9331B78002BECD0CA
:1078D000F8342378012BE8D10020E6E7032089075C
:1078E000FAD4E2E7F0B51F00184B85B01C68019090
:1078F00002910392002C27D1200005B0F0BDA568AD
:107900003301ED186B89019A934211D3029A934285
:107910000ED8002F04D10A9B002B10D12C00EBE7CE
:107920003B002978039A6868FEF7F6FC0028F2D13C
:107930000136B6B2A388B342E1D82468DAE7A36877
:107940000A9A5B891380E9E70026F3E7D866FF1FF0
:1079500037B50C000A8849880123914217D3002AC1
:1079600015D0651D23792A0002210A48FEF7D4FCB0
:10797000102300280BD023796188208800242A0056
:107980000094FFF7AFFF0A23A04200D023001800A5
:107990003EBDC04642BE001113B50A0008884988A2
:1079A000012388420BD8002809D00024137905321E
:1079B0000094FFF797FF0A23A04200D0230018008D
:1079C00016BD13B50A0008884988012388420BD8E0
:1079D000002809D00024137905320094FFF782FFB4
:1079E0000A23A04200D02300180016BDF0B58BB0CA
:1079F00003904A8808880E000123824255D300284C
:107A000053D00023012704AC237000227188130097
:107A10000092FFF767FF051E3ED02078002835D181
:107A20002B78022B18D167706A8983000130E31824
:107A300080005A8069680222201804F0A9F823788F
:107A40000133DBB22370042B19D93B006889013064
:107A500080B2002BD9D01FE0022363701223584359
:107A60006A89231804305A8069681022201804F0AB
:107A70008FF823780133DBB22370002BE5D10C4A59
:107A80006B899B185A425341DBB2DFE76378012BC5
:107A9000E4D12B78022BC7D022780A23002A04D005
:107AA00021000398FEF798F9002318000BB0F0BDF1
:107AB0000100FFFF0F4BF0B504001868002816D036
:107AC00083685D89A54207D88288AE18B44203DA7C
:107AD00012019A18934201D10068EFE71E005F89F6
:107AE0001036A74204D1002900D00D801800F0BD47
:107AF0003300EFE7D866FF1F70B505000C0008885B
:107B00000021FFF7D7FF03000120002B04D0220043
:107B10002800197AFFF7C1FE70BDF7B50C000025EB
:107B200001902300F6331B78AB4201D800200AE015
:107B30006B00E65A00213000E718FFF7BBFF002872
:107B400002D126800130FEBD017A0198FFF794FE34
:107B5000002802D03B882380F5E70135EDB2E0E74D
:107B600010B5040008880021FFF7A4FF03000120DE
:107B7000002B03D02000197AFFF77EFE10BD000015
:107B8000054B1B68002B01D1180004E09A6852894C
:107B90008242F6D198887047D866FF1FF0B50E274D
:107BA000002687B0039302ABFF183E8005001F4BF1
:107BB00040891400984207D02B78013000976A68FA
:107BC00080B2FFF78FFE060002212B7818486A6802
:107BD000FEF7A2FB00280FD06C892000FFF7D0FF32
:107BE000002802D0013C0419A4B2039B002B00D052
:107BF0001C80300007B0F0BD02212B780D486A6868
:107C0000FEF78AFB0028E7D102212B780A486A6830
:107C1000FEF782FB002807D0002EDED03B88A3426F
:107C2000DBD17489013CDFE76C89DEE7FFFF0000F0
:107C300042BE001140BE00113EBE001110B50C0046
:107C4000FFF7DEFC03000220002B0AD0002C00D03E
:107C500023609B781720FE2B03D00138FF2B00D127
:107C6000002010BD73B50D0001A904001600FFF738
:107C7000E5FF172805D0002E04D129002000FEF7CB
:107C800027F976BD01221021200000F047FE0028D0
:107C9000F3D0F6E7014B18607047C046E866FF1F57
:107CA00037B56B469D1D010004000222280003F039
:107CB000F7FE2B88B02B0ED12379122B09D123008C
:107CC000FF339B78012B06D10121608800F0E0F89A
:107CD00001E01B2BF8D037BD10B5054B04211870FF
:107CE00000F098F8FFF74CFDFEF770FB10BDC046A2
:107CF000EC66FF1F0020F0B50BB20F0087B0834287
:107D000034DA274B187803F0A3FC051E2BD0037838
:107D1000A02B25D103AE3100FEF7E4F8041E0BD1F1
:107D2000B378DB0724D51F4B06341B68002B03D028
:107D30003100688898470400A868002801D003F043
:107D40005FFD002C08D1184A039B1340174A934249
:107D500006D0B3781B2B03D00121688800F098F877
:107D6000280003F0FDFB80200002784007B0F0BD42
:107D70000F4B1B68002B10D0310068889847041EF9
:107D8000DAD07378002BD7D1B27801A90A704B8072
:107D90000C716888FDF7F6FFCEE70624F1E7C046D0
:107DA000EC66FF1FE466FF1F00FFFF0000011200EA
:107DB000E866FF1FF7B50190822040000D00170014
:107DC0001E0003F0A5FD04001320002C12D0B023E8
:107DD00020002370089BFC226770658026710830A4
:107DE000002B08D0190003F0D3FE2100019803F006
:107DF00077FE0020FEBD089903F0FAFDF5E710B507
:107E0000041E06D00078FD2803D803F089FDFF2367
:107E1000237010BD0A1F93B210B504000220032B7B
:107E200005D882400020024BD1529B189C7010BD97
:107E30000C67FF1F0B8870B5043B04000D00022087
:107E4000032B0BD80121200000F04CFD030014206F
:107E5000002B03D02900200000F0DEFB70BD0000E5
:107E600007B51300034A00920A00012100F02CFC20
:107E70000EBDC0469D80001107B5019203220092FD
:107E8000024B0A00122100F049FC0EBD1B810011BB
:107E900007B56B4601AA11800449D88008780633DB
:107EA000012802D1190003F0B3FB07BDED66FF1FE7
:107EB0000C4B10B518700023FF210B4A138013815F
:107EC00093819380094A5380137051729381937206
:107ED000D174D3821375517703F072FB00F0FCF973
:107EE00010BDC0461C67FF1F0C67FF1FEE66FF1F1B
:107EF000F0B58DB06B46002003910C229B5E83424F
:107F000000DBB0E05D4B187803F0A2FB051E00D14A
:107F1000A4E00378902B00D09DE006AF01004688D6
:107F2000380000F013FA79680400002900D19CE0C1
:107F30003B88052B6ED13B89032B1CD905AC200057
:107F400000F0A2F86288172A61D83989131D994276
:107F500031D17968237804310291D90738D5607816
:107F600000F08EF9071E06D0002303712378012B41
:107F700008D0132B23D0A868002800D178E003F0A4
:107F80003FFC75E06288029909A800F0A6F802900B
:107F9000380000F08BF909AA2378387A0192002280
:107FA00031000092029A00F012F9380000F064F9F2
:107FB000029B002BDFD0300000F080F9DBE7037874
:107FC000032BD8D16288029909A800F0D6F8DEE721
:107FD000122B13D1029909A800F0B5F8021EEAD1BC
:107FE00027498B88002BC6D0887909A9237801916D
:107FF00061780091310000F0EAF8BCE7002302AAA2
:1080000093833000617809AAFFF72AFFB3E71D4B7D
:108010000993F6E7042B02D09A1F012AABD8184A1D
:10802000043B9B00995A0029A5D0D21890783100C2
:108030003A0000F0AEF800289DD13B88042B03D015
:1080400001213000FFF724FF012C04D1A86800288B
:1080500001D003F0D5FB280003F082FA8020039BB7
:108060000002434018000DB0F0BD012800D182E7A6
:1080700001213000FFF70CFFEDE7C0461C67FF1F32
:108080000C67FF1F010017000B7803704B784370DB
:10809000CB788A781B021343438070470A88030019
:1080A00002700A88120A42700A88012A06D14A8898
:1080B00082704A88120AC2700420704702208242ED
:1080C000FBD14A8804309A704A88120ADA708A888A
:1080D0001A718A88120A5A71EFE710B5040001205C
:1080E00082420CD94B780A781B02134323808342C7
:1080F00006D1CB788A781B0213436380002010BD21
:10810000022BFBD1CB788A781B02134363804B7917
:108110000A791B021343A380F0E70B8803700B88D6
:108120001B0A43704B8883704B881B0AC3708B8873
:1081300003718B881B0A4371CB888371CB881B0A20
:10814000C3710820704703000120082A14D14A781F
:108150000878120202431A80CA7888781202024311
:108160005A804A790879120202439A80CA7988793A
:10817000120202430020DA80704710B5040001208B
:10818000022A05D100204B780A781B021343238072
:1081900010BDF8B5060010200F00150003F0B8FB65
:1081A00004000120002C0ED0A0230C2229002380E3
:1081B0006780201D002D07D003F0EAFC210030006D
:1081C00003F08EFC0020F8BD03F012FCF6E7F7B5D3
:1081D0001E00009008AB142017001D78019103F0D9
:1081E00097FB041E12D0A2230370019B47704380AB
:1081F000099B057146710C220830002B07D019002D
:1082000003F0C6FC2100009803F06AFCF7BD099951
:1082100003F0EEFBF6E737B5041E0FD04388002BC2
:108220000CD00025C1881323007A172201950095F0
:10823000FFF7CDFFFF2365806372257037BD000017
:1082400010B50C4904004A88002A09D08B89002BFC
:1082500005D00020CB8A0222834201D010BD01222A
:1082600013000A20434300204032C854C8184280FB
:108270000472F3E7EE66FF1F00234380037070472C
:10828000094B00211A0010B55C88002C06D01C791F
:10829000844203D10A234B43D01810BD01310A3365
:1082A0000329F1D10020F8E7EE66FF1F10B50400A6
:1082B000407A03F035FBFF23637210BD7047043032
:1082C00010B580B203F024FA002803D004214942FB
:1082D00003F08EF910BD000070B50025104CA068A9
:1082E0002580A581A580A84202D003F089FAA56067
:1082F00000250C4C0C4B606D1D80230058331D7005
:10830000A84202D003F07CFA656500256068002869
:1083100001D003F075FA013508340A2DF6D170BD8D
:10832000B467FF1F5867FF1FA867FF1F70B5041EC3
:1083300009D1054D2880A881A880A868002802D00E
:1083400003F05EFAAC6070BDB467FF1FF0B54B88F8
:1083500085B00193002343600A7905000F00022ACB
:1083600000D07BE0CA88032A17D98B685E78197819
:108370003602DC78D8790E4399781B7A24021B02E6
:108380000C43034353495BBA0B80331D93421ED108
:10839000042C04D0631F022B0ED9012015E0019A92
:1083A0004D4B1201D35A002B06D00198FFF7BEFFA8
:1083B0004A4A1369013313610421B8682E812C8065
:1083C000494203F015F96860002005B0F0BD434D47
:1083D000042C06D0631F022B0FD9EB680133EB602E
:1083E000DBE7019A3C4B1201D35A002B05D00198D0
:1083F000FFF79CFF2B6901332B61374B3000029351
:10840000019B029A1B010193002301998C468B5218
:10841000130063449C8003939E81FFF750FF039BEE
:10842000041E986016D00421B868494203F0E0F8B1
:10843000FA880100043A200003F0AAFB0199029A8D
:10844000FB888A5A043B9B18029A8B522B68013393
:108450002B60A2E7AB690133AB619EE71E4B029331
:10846000019B1E01029BF35A002B2DD002998C19FF
:10847000A068002828D0012A26D1FA889B189BB230
:108480007352A189994217D39B1AC018B96803F097
:108490007FFB029BA289F35A934200D07DE7002222
:1084A0002B81A3882B80A3686B60029BF2520B4A3E
:1084B00053680133536070E7084A9368013393604F
:1084C0000198FFF733FF68E7044A536901335361AA
:1084D000F6E7C0461E67FF1FB467FF1F2467FF1F34
:1084E00070B5051E15D10B4C0B4B1880230058336B
:1084F0001870606D002802D003F082F965652500D0
:1085000050356068002801D003F07AF90834AC4295
:10851000F7D170BD5867FF1FA867FF1FF0B51700A0
:10852000A12285B0920001934243394B06001B689B
:108530000C009B18D933FF331D78FDF741FF043041
:10854000854204DD3000FDF73BFF0430C5B2BD427B
:1085500007D33A0000213000019B03F081F805B0F9
:10856000F0BD2900380003F01BFA2300C6B25033D7
:108570001E700393019B29006365380003F058FACD
:10858000CBB20293002B02D0039B01361E70002653
:108590002300503303931B78B34204D8606D002846
:1085A00031D10020DBE7029A2800002A04D0013BE9
:1085B0001000B34200D02800F700E719387003F02C
:1085C00027FA786000280ED03A78019903F0E0FA93
:1085D000019A3B780136D3180E4A0193D369F6B25B
:1085E0000133D361D4E7039B18706065A74205D1BE
:1085F000084A1320D36A0133D362B0E7606803F0FE
:10860000FFF80834F2E703F0FBF800236365C8E7DE
:108610003409FF1F2467FF1FF7B50D000700042171
:10862000686802F0E5FF2B89040003702B891B0AA0
:1086300043702B8883702B881B0AC3702E890225F8
:108640000436F6B2FB2E15D81B4B9F4214D10C20DA
:1086500003F05EF91135011E0CD0902303708E3BA0
:108660000371043B4380154B8460C680187803F087
:1086700037FA00252800FEBD5C237B43104AD3183F
:108680000093583301931B78002B0FD10300320065
:1086900038000099FFF742FF019B05001B78002B73
:1086A000E8D13800009903F0CBF9E3E7054A072544
:1086B000536A01335362DDE7FEFF00001C67FF1FB2
:1086C0005867FF1F2467FF1FF0B587B00090172081
:1086D0000F0016000193FFF7F2FD1325041E19D0B9
:1086E0000C98031E02D00199201D9847030AE370DD
:1086F000052302AAA070043090812770009866704C
:1087000003A993800494FFF787FF051E02D0200081
:1087100003F076F8280007B0F0BD0000F0B587B090
:108720001F000CAB1B780391059301210DAB0600D4
:108730001C78049200F0D6F81425002821D02000DF
:10874000FFF77EFD0135041E1BD01149059B0A78F9
:1087500003700132D2B2131EC68001D101231A0068
:108760000B7022713000049B03990097FFF7ACFF58
:10877000051E09D1230021000648074A093303F0EA
:10878000DFF9280007B0F0BD002363802370F8E70D
:108790002067FF1F1782001130750000F8B5050033
:1087A0000E00064C064F2368002B02D03100280033
:1087B00098470434BC42F6D1F8BDC046C467FF1FD9
:1087C000D867FF1F0123064A5B42538000231371C1
:1087D0005362044A136053609360D360136170471F
:1087E000D867FF1FC467FF1F0200002310B50649AA
:1087F0009C000859002801D1625010BD0133052B9F
:10880000F6D11320F9E7C046C467FF1F034A538817
:10881000181A43425841404210407047D867FF1F22
:10882000F0B585B002930AAB1F780CAB1B880090A3
:1088300008000E0001920393FFF7E8FF05001120E6
:10884000002D1BD10E48FFF7E1FF04001520002C7E
:1088500014D006220B99A771E01D03F099F9019B32
:1088600030002371029B29006371009B6680237096
:10887000039B6562E381FFF791FF280005B0F0BD1F
:10888000FFFF000010B5FFF7C1FF04000220002C1D
:1088900012D060880121FFF781FF606A002801D0B3
:1088A00002F0DEFF28220021200003F0A1F80123BE
:1088B00000205B426380207110BD000030B5074A84
:1088C000074C5588010013780020A54204D05B1A9C
:1088D00059424B415842104030BDC046D867FF1F37
:1088E000FFFF0000084A10B501230C00904208D099
:1088F000FFF78CFF031E04D0037923405A1E9341D7
:10890000DBB2180010BDC046FEFF0000024B187914
:10891000431E9841C0B27047D867FF1F70B504006E
:108920000D001600FFF772FF002804D10D4B9C428A
:1089300000D0143070BD416A03790520002907D0AA
:1089400012221A40102A02D10520002EF2D10F2047
:10895000DB06EFD5897E0C20A94289414942494274
:108960000840E7E7FEFF0000030010B5002800D133
:1089700010BD0348034A41889142F9D09847F7E770
:10898000D867FF1FFFFF0000002330B5C45CCD5C3B
:108990006C40D4540133102BF8D130BD0F2300228A
:1089A00010B5C45C64002243CA54C25CD209013BC6
:1089B000F7D210BD0200010010B52032103102F0D4
:1089C0002FFE10BDF0B58BB003901020059317005B
:1089D000049102F07DFE0090102002F079FE009BD1
:1089E00013240190002B05D000280CD113240098EB
:1089F00002F036FF019B002B02D0180002F030FF7E
:108A000020000BB0F0BD102002F062FE0600102026
:108A100002F05EFE13240500002E00D1AEE0002817
:108A200019D01022002102F0E3FF32002900039840
:108A300002F0F6FD041E0ED133787F2B51D83000A2
:108A40000099FFF7ABFF009B1B787F2B53D8019950
:108A50000098FFF7A3FF300002F002FF002D02D0C4
:108A6000280002F0FDFE002CC1D1102002F030FEE3
:108A70000600102002F02CFE0290002E7CD0002870
:108A800078D03A000F3223000125121105D00F33A0
:108A90003B4015B25A4253411BB26A1E1201002BD1
:108AA00033D0049BD2B298180099029AFFF76CFF5A
:108AB000013D10220021300002F09AFFADB2049F68
:108AC0002D017D19AF4242D0002C33D0300002F08E
:108AD000C7FE029B002B00D189E7180002F0C0FE00
:108AE00085E729003000FFF759FF28002549009A43
:108AF000FFF74AFFA7E729000098FFF74FFF28007C
:108B00002049019AFFF740FFA5E70F210F40049984
:108B10008A18D9B28F4208D9D15C06A819540133FA
:108B2000102BF6D1029A0199C0E7791A48424141C7
:108B3000C901F2E73900300006AAFFF725FF32002D
:108B4000039806A902F06CFD10370400BAE7002C68
:108B5000BCD13000029906AAFFF716FF320006A921
:108B6000039802F05DFD082204003100059803F02F
:108B70000FF8ABE71324A9E71324AAE7002800D0D5
:108B80006EE733E748BE0011F0B58BB00F0016005A
:108B90000225009000283FD0002A3DD00B1DDBB2FB
:108BA0001800029302F094FD1135041E34D0FDF735
:108BB00047FD05003A000099201D02F0A1FEEBB22E
:108BC0000393E3702B0CDBB22F0A00936370FFB2A8
:108BD0002B0E2370A7700193FDF72CFD10220100CE
:108BE00006A802F08DFE2100029A04AB06A8FFF74A
:108BF000E9FE051E0DD1039B08223370009B04A9DA
:108C0000B370019B7770F370301D02F079FEFDF7B1
:108C10001DFD200002F024FE28000BB0F0BDF0B5D1
:108C20008FB00D00149E039004920593002A03D187
:108C3000022420000FB0F0BD002EF9D00398FFF7FA
:108C4000E5FD1424071EF4D07278337812021A431B
:108C5000B3781B041343F27812061A43036A019295
:108C6000934201D30133E3D1002D03D03B7901249A
:108C70009B07DED50822002106A802F0B9FE059B5D
:108C800013240433DBB21800029302F021FD051E09
:108C9000CFD0059A0499043002F032FE042231004C
:108CA000280002F02DFE3900102210310AA802F02F
:108CB00027FE2900029A06AB0AA8FFF783FE041ECE
:108CC0000FD1082206A908A802F01AFE0822311DB9
:108CD00008A802F0CDFE012807D101990398FDF7FD
:108CE000C9FC280002F0BCFDA3E70124F9E700005D
:108CF00070B51C4C05002368181E10D0002D14D12F
:108D00001A78002A0CD1981C083202F041FF02F0B8
:108D1000A7FE0135002808D123681D70012070BD11
:108D20000A331800082202F033FF2368002BF5D025
:108D3000122002F0EDFD061E0DD0C1232168037044
:108D4000457002311022023002F022FF2368310008
:108D5000587802F0C5FE206802F082FD00232360EF
:108D6000DCE7C0460068FF1FF8B504002020FDF7CF
:108D700055FB0D4EA700BB590500002B0DD0002858
:108D80000BD0D878FF2809D108492A000C55F3598F
:108D900007480333611802F0D3FEF8BD290002F042
:108DA000DFFC0028F0D1F8E71C68FF1F0468FF1FF4
:108DB000C19F001170B5064D84006359002B05D08A
:108DC000D87802F0ADFDFF226359DA7070BDC0465D
:108DD0001C68FF1F70B506008CB00C001500002148
:108DE0003022684602F004FE31001022684602F08C
:108DF00087FD1D2021000322684402F081FD6846A2
:108E0000FFF7D8FD2D21040003222800694402F059
:108E100077FD20000CB070BDF0B50700160097B0CC
:108E200001931CAB1D7830221EAB00910AA80021D3
:108E30001C7802F0DDFD102239000AA802F060FD66
:108E40001022002102A802F0D3FD0722310002A85F
:108E500002F056FD072202AB9818631E9C4101994F
:108E600002F04EFD02AB9C732B005A1E934102AAE6
:108E7000D3730021102206A802F0BAFD06221D9924
:108E800007A802F03DFD1A2002ABC01806221F9968
:108E900002F036FD102200990EA802F031FD1022DA
:108EA00002AB0EA908781C78013A6040D2B2087073
:108EB00001330131002AF5D10AA8FFF77BFD10220A
:108EC00012A904000EA802F063FE102206AB0EA940
:108ED00008781D78013A6840D2B208700133013138
:108EE000002AF5D10AA8FFF765FD04431022209857
:108EF000E4B212A902F004FD200017B0F0BD70B575
:108F00000E0014008CB00100102268461D0002F013
:108F1000F7FC3100082204A802F0F2FC210008222C
:108F200006A802F0EDFC6846FFF744FD040010229D
:108F3000280008A902F0E4FC20000CB070BDF8B5D0
:108F400006000D0000243719AC4200D3F8BD02F032
:108F500017FB030A3B70631CDBB201379D4203D948
:108F60000234F054E4B2EEE71C00EDE773B50600FE
:108F70000C000225002819D0002917D0032101A8D0
:108F8000FFF7DDFF6B469A793F231A400133134305
:108F90006A463000937101A92200FFF71BFF051EEE
:108FA00004D10322E01C01A902F0F2FD280076BDE5
:108FB00003785807DA08C00FD20080009B071043DF
:108FC0009B0F1843C0B2704707230B40C908C90064
:108FD0000B4303707047000070B50400FFF7EAFE12
:108FE000134DA4006359002B21D0186A002801D02A
:108FF00002F036FC2B59986E002801D002F030FCAC
:109000002B59D86E002801D002F02AFC2B59186F7A
:10901000002801D002F024FC2B59586F002801D001
:1090200002F01EFC285902F01BFC00232B5170BDDE
:109030001C68FF1F0E4B8000C35870B50C00002B3E
:109040000FD09D68002D0CD02B78201D0B706B78F5
:109050004B70A97CFFF7B8FF2B7E23726B69E3602E
:1090600070BD10220021200002F0C2FCF8E7C046CB
:109070001C68FF1F014B18607047C0461868FF1F2F
:10908000074A03008000825810B5002A06D0D08815
:10909000984203D1012901D1FFF79EFF10BDC046C0
:1090A0001C68FF1FF0B5264E95B087000B93BB5987
:1090B0000500099112200A92002B31D0D888FFF7C1
:1090C000A5FB04001420002C2AD0280010A9FFF7CB
:1090D000B1FFBB591E781D6A002E23D00895FDF7FD
:1090E000EFFA07000020FDF7F1FA0790A379E61DDB
:1090F000069310AD0CA9089800F0E2FA0EA928001A
:1091000000F0D7FA0B9B0A990493069B09980293E7
:10911000079B0396019300970EAB0CAAFFF77CFE0A
:1091200015B0F0BDFDF7CCFA06903000FDF7CEFA91
:10913000E31DA779079310AB06000893DAE7C04652
:109140001C68FF1F30B50C4C85002A59030085B000
:109150000120002A0ED018006946FFF76BFF2B593B
:109160001A78D888054B002A00D1054B6A4607219A
:1091700000F0D9FB05B030BD1C68FF1FB39600118D
:10918000C196001130B5094C8500295985B01022CF
:109190006846253102F0FCFC2A591121044BD08885
:1091A0006A4600F0C0FB05B030BDC0461C68FF1F1A
:1091B0005D97001130B5094C8500295985B0102202
:1091C0006846353102F0E4FC2A591121044BD0885D
:1091D0006A4600F0A8FB05B030BDC0461C68FF1F02
:1091E0009B970011F7B54D4F86001020F4590D00E4
:1091F00002F06EFAF3592062186A132200286CD02C
:10920000033A29009C6802F0C3FCF3591A780192D2
:10921000002A58D11E6A227D317B9446514001229A
:10922000019F114201D167461740217D9143394387
:109230002175377B4F40BC4660460027800701D42C
:109240004F081740012102208F40227D82433A437C
:109250002275377B5740BC4660460027400701D443
:1092600097080F400420227DBF0082433A432275B5
:10927000627D002794466046727B42400A4201D1DB
:1092800067460F400121627D8A433A436275777BCE
:109290005740BC4660460027800701D457080F405E
:1092A0000220627D7F00824317436775767B002230
:1092B0007E40760701D4BA080A400426617D9200F8
:1092C000B1430A4362756A78002A08D06278002A9E
:1092D00005D005220533DA7700221000FEBD0422F6
:1092E0002979114205D1A17C114202D10533033AFB
:1092F000F1E7019A21782C78002A02D10A00210096
:10930000140018220429E8D8042CE6D8052060436C
:10931000034A05331218525CDDE7C0461C68FF1F84
:1093200058BE001110B50A001121024B00F0FBFAE3
:1093300010BDC046F79700110B0030B587B001ADE6
:109340002B806B4604001100981D082202F020FCBF
:109350002A000B212000024B00F0E5FA07B030BDD7
:109360001F98001110B50A001121024B00F0DBFA22
:1093700010BDC0467398001113B50B0011006A466A
:1093800013706B4604000622581C02F001FC6A466A
:1093900008212000014B00F0C6FA13BD939800117C
:1093A00010B50A001121024B00F0BDFA10BDC046F5
:1093B000E39800117FB505000B4BAA00D4580800B4
:1093C000002C0FD0666F237FE28821780396266FEA
:1093D0000296E66E0196A46E0094FDF709FC280043
:1093E000FFF7FAFD7FBDC0461C68FF1F10B51721AF
:1093F000FFF7E0FF10BD000070B50A000D00064B3E
:109400000221040000F08FFA060029782000FFF7FF
:10941000D1FF300070BDC046C397001170B586B053
:1094200000236A461370836804001D78681E0A28AA
:1094300059D801A902F0F4FA060633373B3F4347F7
:109440004B4F5300180000F042F9062312284BD06E
:1094500000281BD16088FFF7D9F90823002813D012
:109460004279002A47D1264B1A78072312070BD5D9
:10947000244B1A680723002A06D01668002E03D052
:10948000290001AAB04703006A4613706B461B7897
:109490006088002B2AD1FFF767FC06B070BD18006A
:1094A00000F06CF9D4E7180000F087F9D0E7180055
:1094B00000F093F9CCE7180000F0ADF9C8E7180008
:1094C00000F0C3F9C4E7180000F0F6F9C0E718008F
:1094D00000F0F6F9BCE7180000F013FAB8E718003E
:1094E00000F013FAB4E707236A46137069466088F0
:1094F000FFF782FFD1E70523012AC5D1024BB8E768
:10950000A966FF1F1468FF1F1868FF1FF8B52C4FCE
:109510008600F35904000D00002B40D0DA88824207
:109520003DD15A78062A33D11A78002A2ED001204C
:1095300099681A6A097D014206D0157B054203D05D
:1095400007225A700120F8BD0220014204D0157B89
:10955000054201D00922F4E70420014204D0127B25
:10956000024201D00B22ECE7164B1B68002BE9D01E
:109570005B68002BE6D020009847BB5900215B7840
:10958000122BDFD12000FFF715FFDBE70E4BECE7D6
:10959000112A04D1002900D032252900F2E7002D3C
:1095A00008D12000FFF732F9002803D010230279F8
:1095B0001343037121002800FDF798FAC2E7C04663
:1095C0001C68FF1F1468FF1F1868FF1F70B50E4E40
:1095D0008500AB590400002B13D01B78002B11D150
:1095E0000A4B1B68002B04D05B68002B01D02000C5
:1095F000984773595B78122B03D100212000FFF7A5
:10960000D9FE70BD024BECE71C68FF1F1868FF1FF6
:109610001468FF1F094B8000C3581020002B0CD08A
:109620001A6A002A09D09B68002B06D0127A1B7E8A
:10963000101C9A4200D9181CC0B270471C68FF1F4A
:1096400070B503000D0014000220002A30D000295C
:109650002ED013700B78081D53704B789370FFF762
:10966000A7FCE070012002212B7A23716B7B034061
:1096700063716A7B0A401343042263716E7B164058
:10968000334363716E7BF608F600334363712B7BC3
:109690000340A371287B014000200B43A371297B69
:1096A0000A401343A3712A7BD208D2001343A3714B
:1096B00070BD10B50A0001000120FFF7C1FF10BD09
:1096C00010B50A0001000220FFF7BAFF10BD70B507
:1096D00006000C000220002E30D000292ED0737816
:1096E000201D0B70B3784B70F178FFF76DFC0122F1
:1096F0003579257271794B10080013409340104062
:109700000343881010408000C9080343C9000B437D
:109710006373B1794B10080013409340104003432A
:10972000881002409200C9081343C9000B4321204E
:109730002373FCF773FE854201D2122070BD2220F4
:10974000257AFCF76BFE8542F7D823781820042B86
:10975000F4D86378012BF1D80020EFE7030010B5AF
:109760000220002909D0002B07D00322481C0A70D0
:1097700019000D3202F00CFA002010BD0300022285
:10978000080010B5002B06D0002904D00E32591C59
:1097900002F0FEF90022100010BD030010B50220F7
:1097A000002909D0002B07D00422481C0A70190098
:1097B0000C3202F0EDF9002010BD10B5FFF7DEFF0E
:1097C00010BD03000220002906D0002B04D0052282
:1097D00000200A701B784B70704703000220002B9A
:1097E00008D0002906D05B7800200B70013B082BC5
:1097F00000D918307047030010B50220002909D0A5
:10980000002B07D00622481C0A7019000A3202F009
:10981000BFF9002010BD10B5FFF7B0FF10BD02006A
:109820000B00022010B500290ED0002A0CD0072111
:109830001970118859701188090A99701118082235
:10984000D81C02F0A5F9002010BD03000A00022078
:1098500010B5002B0CD000290AD09978587809024D
:1098600001431180901CD91C082202F091F90020BC
:1098700010BD030010B50220002909D0002B07D02D
:109880000822481C0A701900921802F081F9002081
:1098900010BD02000B00022010B500290BD0002AD9
:1098A00009D009211970117818185970511C062215
:1098B00002F06EF9002010BD10B5FFF75FFF10BD7C
:1098C00002000B00022010B5002A09D0002907D0A1
:1098D0005178197011180622581C02F059F900200D
:1098E00010BD030010B50220002909D0002B07D0BD
:1098F0000A22481C0A701900063202F049F90020B9
:1099000010BD10B5FFF73AFF10BD02000B0002209A
:1099100010B5002A06D0002904D018005178FFF7AE
:1099200053FB002010BDF0B585B017001E006A463D
:1099300006230500080091819380FEF7C0FC1324E4
:10994000011E02900CD03800B047041E05D128003B
:1099500001A9FEF76FFA041E02D0029801F050FF31
:109960002800FFF701FA200005B0F0BDF0B50400B3
:109970008BB0019115000021102202A802F038F8E6
:10998000334EA700B85900283CD0C388A34239D130
:109990000378002B36D14278062A18D10200010044
:1099A000553235310C3006ABFFF7A9FA002829D122
:1099B0002000FFF72FFE020006A902A802F0E8F837
:1099C000200002A901F0F4FD01200BB0F0BD816E72
:1099D000002917D00B8A112A28D19D420ED1019857
:1099E0001231093A02F044F8012807D1BB5920008E
:1099F0009D6EFFF70FFE29000200DEE732212000F6
:109A0000FFF7D8FC2000FEF701FF061E1BD0416ABD
:109A1000002918D00B8AAB4215D1082201981231C7
:109A200002F026F801280ED1716A0AE09D42E9D1C0
:109A300008220198123102F01BF80128E2D1BB592B
:109A4000996E8A7EB9E7200001F062FDBCE7C0464E
:109A50001C68FF1FF0B56B4D87007E5985B03378C9
:109A600002900393002B00D087E0B368346A01931F
:109A70007078062817D101221B7D134202D0217B6A
:109A8000114218D10222134202D0217B114251D13E
:109A90000422134203D0237B134200D08BE0019BAE
:109AA0005A7DEB5991E007380428F8D801F0B8FF47
:109AB000032E42678300B36E002B03D11C2001F0FC
:109AC00007FEB066EB599C6E002C1CD010220021C2
:109AD000200001F08DFF0298FFF79CFD010020009F
:109AE000FFF72DFA01F04CFD2082200008211230F2
:109AF000FFF725FA0298FFF78DFDA076EB592100BC
:109B0000D888FFF70FFC0822EB591CE0B36E002B3E
:109B100005D01A00198AF0881232FFF70DFC0222D4
:109B2000019B197DEB5911423DD0207B10423AD068
:109B3000073208E0F488FCF7DBFD01002000FFF7A6
:109B400011FC0A22EB595A70029B9C002A59537847
:109B5000073B042B11D8D088FEF758FE00284ED0C2
:109B6000C3895A08D2182849029B0298CB542B5912
:109B700041180433254801F0E3FF05B0F0BDFCF7C0
:109B80009FFD03000120834201D100200393EB5984
:109B9000DE88FCF79BFD039902003000FFF7ECFB29
:109BA000019AEB59117D042211420CD0217B114204
:109BB00009D00B22C7E7F688FCF73CFD0100300016
:109BC000FFF7EEFB6BE7019A527D01210A4204D0B8
:109BD000607B084201D00C22B5E702210A4204D082
:109BE000607B084201D00E22ADE704210A4204D076
:109BF000627B0A4201D01022A5E71222A3E7FA22D3
:109C00005200B0E71C68FF1F2068FF1FCB9F0011A8
:109C100010B5064B1A780423100018401A4200D0E1
:109C20000348FFF727FA002010BDC046A966FF1FB2
:109C30002C45FF1F70B50400FFF7D4FA051E43D171
:109C40002000FFF77FFA234EA400A0598268937C7E
:109C5000DB0708D50321036A1B790B40012B02D1D6
:109C6000017F0B430377431DD97F8B1E022B0DD839
:109C7000022900D00121C088FCF790FF042133594C
:109C80001A7F59700A431A77280070BD01290CD138
:109C900002231022437000210C3001F0A9FE30593C
:109CA00010213530FFF74BF9EEE70529ECD10223FF
:109CB000D118437010220C3001F06AFF042332598E
:109CC000117F0B431377EAE708251828DCD1053DFF
:109CD000DAE7C0461C68FF1FF0B58BB005914388DA
:109CE0007E4F9E00F45915000493002C15D10129D4
:109CF00002D000200BB0F0BD101D57781678FFF78A
:109D000057F9EB68320002932B7A04990193009083
:109D10003B002000FCF70CFFEBE7E388049A93423A
:109D200001D00820E6E72378012B00D1D4E0059B81
:109D3000581E092800D9CFE001F072FE05CE0A298D
:109D4000CC506C859AB229000498FFF773FFD1E7D5
:109D5000200029001022453001F01AFFB9594B7834
:109D6000042B02D1013B4B70C3E70B000A002533E3
:109D700035320C310498FFF795F90498FFF702FA91
:109D80000522431E9841BB59C0005A70B2E720001B
:109D900029001022553001F0FBFE049B4F4C9D0022
:109DA000295904980A0006AB55320C31FFF77AF9AD
:109DB00029591022453106A801F05AFE012808D180
:109DC0000498FFF7F7F90590002804D106222B59D3
:109DD0005A7005988EE708230593FAE763780C2BF1
:109DE0007AD1E36E002B03D11C2001F071FCE066F8
:109DF000BB59D86E00286FD01022290001F0C8FE90
:109E0000BB590498DC6EFFF705FC0D22A076BB5908
:109E10005A706EE7E06E00285ED063780D2B5BD140
:109E20002B8808220382A91C123001F0B1FEBB5915
:109E30009A68517D0222114226D0186A407B104256
:109E400022D00C32E4E763780E2B45D1236F002B30
:109E500003D1162001F03CFC2067BB59186F002885
:109E600003D01022290001F093FE0F22BB59CFE747
:109E700063780F2B30D1206F0622691C103001F05F
:109E800087FEBB599A68517D0422114203D0196A9A
:109E9000497B1142D5D100210498FFF78BFA28E7BE
:109EA000636F002B0DD0BB59586F0028F3D01022E0
:109EB000290001F06DFE0122BB5952425B6F1A610D
:109EC000E9E7142001F004FCBB5960675B6F002BCD
:109ED000E9D126E72978DFE707200BE71C68FF1F99
:109EE00010B5064C207001F033FE06212078FDF7F6
:109EF00091FF0348FEF778FC10BDC0462F68FF1F96
:109F00008190001100200BB270B50D00834216DA6B
:109F1000264B187801F09CFB041E0DD00378922B81
:109F20000ED0A02B37D0224B1878FF283AD0210032
:109F300001F0D6FD002835D180200002684070BDB8
:109F400043780E2B0BD03E2BEDD18378052B12D00E
:109F5000082BE8D181798088FFF7D8FA08E0154B03
:109F600082889A42DFD183681878591CFEF7C0FEB8
:109F7000002817D1D7E7104B1B785B0712D50F4B82
:109F80001B68002B0ED09B68002B0BD0C289811D53
:109F900080889847ECE7FFF741FAA068002801D0D5
:109FA00001F02EFC200001F0DBFAC5E72F68FF1F4F
:109FB0002545FF1F18200000A966FF1F1868FF1F16
:109FC00010B50078FFF712FA10BD10B50078FFF752
:109FD000FDFA10BD0C234343084A10B59B185A687C
:109FE000002A03D0012901D1904710BD9B68002BA6
:109FF000FBD00029F9D19847F7E7C0464C68FF1F0E
:10A0000010B5162813D801238340094A946B1C43CA
:10A010009463506B98435063D46B2000984301299C
:10A0200001D120001843D063116B0B43136310BDA3
:10A0300000800040F0B500240127154B85B0DA6B95
:10A04000144E03921A6C0192DA64019BE3403B4286
:10A0500017D0039DE5403D400295E5B202992800E6
:10A06000FFF7B8FF316A736A002908D03900002B66
:10A0700001D0029979402800FFF7C2FF01E0002BD0
:10A08000F9D101340C36172CDFD105B0F0BDC04634
:10A09000008000403068FF1F10B50124020020003E
:10A0A000162A08D8054B5968D140214204D01868B7
:10A0B000D0400123184010BD186DF9E70080004022
:10A0C000162807D80122064B8240002903D0D96800
:10A0D0000A43DA607047D9689143D960FAE7C0460D
:10A0E0000038004030B5162818D8032444430F4BDD
:10A0F000E25C1B199C785D7801232D1B0135AB4078
:10A10000013BA340A140DB430C00122807D80849BB
:10A1100092005218116819402143116030BD054A60
:10A1200011680B4023431360F8E7C0469FBE00113F
:10A1300008F0004014F00040C21F70B5D4B20623EE
:10A14000092C0BD80125084C9540002908D0002186
:10A15000FFF7C8FF23682B4323600023180070BD5E
:10A160002368AB43F8E7C04600380040F0B5162836
:10A1700026D8214B1B185B78022B21D103244443A2
:10A180001E4A1F4EA35C12199478012215008540C7
:10A19000B76B013CE4B23D43A240B563194C1228B1
:10A1A00015D89B0000290CD117495B1899680A4300
:10A1B0009A600123205C154A834011680B431360A9
:10A1C000F0BD11495B18996891439960F1E70E4B16
:10A1D00000290DD159690A435A61225C1328E8D03D
:10A1E0000123203A93400A49086803430B60E7E7DC
:10A1F000596991435961F0E73068FF1F9FBE001114
:10A2000000800040E4BE001100F00040A0F00040DB
:10A21000A4F00040F8B500241B4E1C4D1C4B1B5DE8
:10A22000012B1FD1184A9269E2401A420BD0012239
:10A23000AA5693402200143AD2B2022A09D81549EC
:10A240004A6913434B6101340C360235172CE5D1B2
:10A25000F8BD0022AA560F499200521891680B438C
:10A260009360F0E7022BEED1E7B23800FFF714FF5E
:10A2700001235840C1B23800FFF778FF3800FFF7DC
:10A280000BFF7077DFE7C0463068FF1F71BE00111B
:10A290003168FF1F00F00040012202388240054B68
:10A2A000002903D059690A435A617047596991439B
:10A2B0005961FAE70038004070B504000D00052030
:10A2C000162C1AD800212000FFF7FAFEA31E012B3E
:10A2D00003D801212000FFF7DFFF00212000FFF756
:10A2E0002BFF01220A49A2400A4B4868012D05D1E3
:10A2F00002431B194A605D70002070BD90434860A6
:10A3000002211C196170996991439961F4E7C04673
:10A31000008000403068FF1F10B516280AD80122BF
:10A32000074B8240002906D019680A431A600121B0
:10A33000FFF7C2FF10BD196891431960F7E7C046E7
:10A340000080004070B505000520162D17D80C239D
:10A3500000246B430A4A21009B181C70094B2800FB
:10A360005B195C70FFF7A8FF0123AB402000064992
:10A370000A681A430A6005490A689A430A6070BD70
:10A380004C68FF1F3068FF1F348000403080004061
:10A3900070B504000E00FF2813D003250540FFF719
:10A3A000D1FF084AA3089B009B183F22ED00AA405A
:10A3B000AE40196820009143314319600121FFF735
:10A3C0007FFE70BD18380040F8B505000520162D39
:10A3D00025D80C246C43124BE4186368002B03D17E
:10A3E000A3680D30002B1AD0022201270D4B00214B
:10A3F0005B195A7028002770FFF75EFF63681E1E06
:10A4000008D0A3683E00002B04D02800FFF744FECC
:10A410004640F6B228003100FFF7F2FD0020F8BDFB
:10A420004C68FF1F3068FF1FF7B5C420FF222B4B7D
:10A4300080001958002491437F3A0A431A50802221
:10A44000274F5202274E1A60274B1D5D002D21D049
:10A45000A31E012B03D80121E0B2FFF71DFF012D40
:10A4600018D11F4B9B69E3402B4213D0E3B2180075
:10A470000193FFF711FE01000198FFF74DFFE3B2D2
:10A48000143B022B1DD801217156184A8D40536987
:10A49000AB4353613B7F002B0DD0E5B22800FFF7A3
:10A4A00093FF2800FFF7F8FD7B7F0100834202D075
:10A4B0002800FFF78FFD01340C370236172CC3D16B
:10A4C000F7BD012100237156F3568D40074A9B00CA
:10A4D0009B189A68AA439A60DCE7C04600E100E056
:10A4E0003068FF1F71BE00113168FF1F00F000408F
:10A4F00010B504000520162C0CD801212000FFF710
:10A50000DBFE0123044A002011194B70A34091691E
:10A510000B43936110BDC0463068FF1F70B50E003D
:10A5200015000400FFF70EFF0C236343094A2000C7
:10A530009B189D605E60FFF747FFF021064B074ABE
:10A540008900051E5A5002D02000FFF7FBFE2800AC
:10A5500070BDC0464C68FF1F0000FF1F35A00011F2
:10A5600070B5134D07202C78002C1FD198222100A4
:10A570005200280001F084F80123C420FF222B7030
:10A580000C4B80001C635C630B4B1C605C600B4BD2
:10A59000195891437F3A0A431A50802252021A6096
:10A5A0000D20074A074901F0BBFA200070BDC046E4
:10A5B0003068FF1F00800040A0F0004000E100E094
:10A5C00029A4001115A20011030010B50620072BC5
:10A5D00009D8054A137001F06BF8D7210020034B0E
:10A5E000034A89005A5010BD5445FF1F0000FF1F49
:10A5F000151BFF1F70B51D0002240C2910D8094A35
:10A60000CA40D2070CD5FBF715FF041E08D1059AE6
:10A6100004992800FBF72AFFFCF798FDFFF7F8FAEA
:10A62000200070BD1210000030B50D7802232C0000
:10A630009C43184201D02B431C0008252300AB4348
:10A64000284201D02B00234320241D00A543204293
:10A6500001D01C4325002A230D70184204D0117824
:10A660001E3B0B43137030BD0028FCD10C21137826
:10A670008B43F7E7F8B51D0006AB1B88140007AA4B
:10A680000E000B201778002B27D10A78022A49D117
:10A690004A68507811780002244A08438018042838
:10A6A00040D801F0BDF903121D1B2300F06801F032
:10A6B000DFF8021CC0B2B84200D93A1CD2B2200066
:10A6C000F1682A8001F064FA06E00222F3681B8830
:10A6D0002A8023701B0A63700020F8BD0622EEE773
:10A6E00001232B80F3681B782370F5E7F368002BB8
:10A6F00016D008222A801A8822701A88120A6270DC
:10A700005A88A2705A88120AE2709A8822719A882E
:10A71000120A6271DA88A271DB881B0AE371DBE737
:10A720002B80D9E701202B80D7E7C04600D6FFFF5A
:10A73000F7B516000A781D0008AB1F880C0001232E
:10A74000022A18D14A685078117800022B4A08432F
:10A75000801803280FD801F063F902254439E06816
:10A7600001F086F8C0B20723B84204D37B190193E5
:10A77000152B02DD0D231800FEBDE0682A00310014
:10A78000C01901F005FA6B4600209B88E268D0549E
:10A790001B4B1B68834203D01B68834200D0984741
:10A7A0000023E8E70B23002FE5D1022DE2D17378D7
:10A7B00032781B021343E2681380114B1B68002B95
:10A7C000EED01B68002BEBD00120E8E70B23002F15
:10A7D000D1D1062DCED12A003100E06801F0D8F9A0
:10A7E000DEE70B23002FC6D1012DC3D1327875339C
:10A7F000012AC0D8E3681A70D2E7C04600D6FFFF2E
:10A800003C6AFF1F70B50C001500072837D801F00F
:10A8100007F9041436361B36242E182015290BD8B8
:10A82000184E16220021300001F0E2F82200290023
:10A83000300001F0ADF9002070BD18200229FBD1D5
:10A840001288114B1A80F6E718200829F4D10A0063
:10A850000E48290001F024F9EDE718200129EBD179
:10A860000B4B10780B49DA69FFF7DEFEE3E718209F
:10A870000129E1D1064B10780749DA6BF4E7022091
:10A88000DAE7C046246AFF1FD245FF1FC845FF1FF5
:10A890005845FF1F8045FF1FA045FF1F030010B54F
:10A8A0000020DB0704D50721024A034800F08CF89A
:10A8B00010BDC046FCBE00115845FF1F054A0300ED
:10A8C0001068002803D082889A4201D180687047BE
:10A8D0000068F6E7406CFF1F0A88030008009A42F0
:10A8E00004D08A8804309A4200D0002070470000CB
:10A8F000F8B5F82200230D4F0D4E7968050042434C
:10A900003370994200D07B600A4C0021200001F096
:10A910006FF800231A007C60AB4202D10020337034
:10A92000F8BD01332280DBB2F834F5E7406DFF1F3C
:10A930003C6DFF1F446CFF1F73B56B460190060012
:10A94000684615001980FCF733FF041E11D1002D55
:10A950000FD07689002E11D00C2000F0B9FE00280F
:10A960000ED0084A0460136886808560002B02D1EF
:10A970001060200076BD1A001B68F7E70224F8E794
:10A980001324F6E7406CFF1F012100220A4B10B58B
:10A9900049420A4C198099809A719A70084B20702C
:10A9A000012019805A60FFF7A3FF2078FCF75EFFB3
:10A9B0000448FDF719FF10BD446AFF1F486DFF1FD3
:10A9C000406DFF1F75AA0011022310B5002802D0A8
:10A9D000FFF7B2FF0300180010BD0000030010B520
:10A9E0000020DB0704D50421024A0348FFF7A4FF37
:10A9F00010BDC04610BF0011D845FF1FF0B50E2690
:10AA000087B003930CAB1F8802ABF6180500080053
:10AA100031000292FDF74EF804000120002C0FD007
:10AA20003088FFF74BFF03000E20002B08D05E6834
:10AA3000002E05D021002800039B029A0097B04702
:10AA400007B0F0BD0A4B10B5984207D10122002390
:10AA500052420A808B708A808B7110BDFFF73CFFD9
:10AA60000028FAD001235B42038000238370F4E7BF
:10AA7000FFFF0000F8B5050001290AD1134E00249C
:10AA80003388F827AB4219D028001149FFF7DAFFC5
:10AA900006E0022904D10139FDF724FF0028EDD09A
:10AAA000F8BD3B0063437268D018D35A002B09D01D
:10AAB0003A00002100F09CFF0134E4B2054B1B7802
:10AAC000A342EED801235B423380DDE7406DFF1FD8
:10AAD000446AFF1F3C6DFF1F10B5FFF7FDFE03002A
:10AAE0000020834200D0987810BD0000F0B589B0F6
:10AAF0001C000EAB80CB03901E8810AB1B78049219
:10AB000002930B7A0D00DB0616D42B780593022BEB
:10AB100024D00498FFF7D2FE002812D003689C4688
:10AB2000002B0ED0029B2200019329003B006446BB
:10AB300003980096A04705E00498FFF7BFFE0028A1
:10AB400002D10E2009B0F0BD8368002BF9D00A2293
:10AB50002900039898470028D7D0F3E76B68587806
:10AB60001A786B4B000210439842D2D8043B9842AB
:10AB700010D2684B984242D015D8674BC0180128B4
:10AB8000C7D80B20002EDDD1EB681A7859683A80BF
:10AB9000200028E0614BC018032800D979E000F0BC
:10ABA0003FFF846A789E5E4B9842B2D10B20002E04
:10ABB000C8D101233B80EB6831001B782370688982
:10ABC000013080B2FCF776FF3A88031E0ED0017880
:10ABD00002328A183A80428962704289120AA2704F
:10ABE00059680278E01C00F0D3FF06E004323A8096
:10ABF00031000422601C00F0FBFE0020A2E70B20C5
:10AC0000002E9FD1EB6807A91E8804233B80330ADE
:10AC1000300026706370FCF74DFF051E28D004AB92
:10AC20009A890E2304A95B183E49C668FCF7B6FF53
:10AC300000280BD12B783C486A680599FBF76CFB20
:10AC4000002803D1012304AA5B42D3813278022A6F
:10AC500006D17168201D00F09BFF3B8802333B80CA
:10AC60000E2304AA9B181B88A3701B0AE370C4E779
:10AC700004ABDE81F4E70B20002E00D062E7E96828
:10AC80000398FFF729FF02233B802070000A6070C1
:10AC9000B3E70B20002E00D054E70222EB681B889C
:10ACA0003A8023701B0A6370A7E7E86800F0E0FDB4
:10ACB000C2B203000720B24200D243E70DD002998E
:10ACC000DBB27118994202DB921BD3B20293029B52
:10ACD000E9681A003B8089195AE70023F6E70B2040
:10ACE000002E00D02EE70722EB683A801A782270F7
:10ACF0005A7862705A88A2705A88120AE2701A79D9
:10AD00002271DA886271DB881B0AA37175E7C0467D
:10AD1000042900000228000000D8FFFFFFD6FFFF33
:10AD200003280000FFFF000040BE0011F0B58DB009
:10AD30006B460020089120229B5E83423DDAA64BA1
:10AD4000187800F085FC071E32D00378B02B2CD188
:10AD50000079023816281FD800F0D2FC17001E0018
:10AD60001E001E0031001E0096001E001D011E0068
:10AD700052011E0073011E00CD011E0050021E0074
:10AD80001E001E008E021E00E302944B94491B8895
:10AD900078880B80FBF700F83800FCF781FF914BB7
:10ADA0001B68002B01D038009847380000F0D8FB12
:10ADB0008020089B0002434018000DB0F0BDF62231
:10ADC0000021874800F014FE0BAA3B7B7989388963
:10ADD00000923A000D32FCF785FD0400804B1B7891
:10ADE000002C3FD146E0804B788805937F4B410093
:10ADF000CB5A0BAE073BDBB23288029300230193A0
:10AE00007B4B210006930093059BFFF76FFE744D6B
:10AE1000002810D1069B3A8A1B889A420BD1380031
:10AE20000599123000F024FE002804D02B786289A6
:10AE30009B00EB185A80162306A81B1832882000A6
:10AE40007989FCF7ABFE2B7804009A00AA18518888
:10AE50000029C3D00133DBB22B70002807D006A92C
:10AE6000C98A9180634A12889A42BCD802E00121C3
:10AE700049429180002B04D059497888FAF7C0FFE5
:10AE80008AE73E890A2479E000253E89574B0693DC
:10AE90007B88069A5B009B5A033B9D4202DB002D98
:10AEA000F0D05BE0162206A812183B7B798900924D
:10AEB0003A0030000D32FCF715FD0590002858D0FF
:10AEC0004689017A7888FCF7D7FC041E44D1464BAA
:10AED00078880793069B4100C95A454B0439C9B28B
:10AEE00006AAD28A06930291019400930599079BC2
:10AEF000FFF7FCFD041E2FD1069B39491A88931CCD
:10AF0000002D26D14B807988384B4900CB5A5119F6
:10AF1000033B8B4220DD059B31485B8941190B7156
:10AF2000A91C0135C9B2EDB2059145191B0A2B7157
:10AF3000059B2D490433181800F02AFE2C4B059A66
:10AF40001B88D318DDB22C4B9E4205D00136B6B219
:10AF50009CE749889942D6D0002D0CD0204C28007F
:10AF6000618800F035FD207021007888FAF758FFDD
:10AF700012E7059CF0E7002C00D183E77B78142BC7
:10AF800000D109E716493B794E800B700C71788827
:10AF9000FAF7F8FE00E7162406ABE418210038891A
:10AFA000FCF788FD011E00D1B7E1788822880F4C9C
:10AFB00045002C5B0A4D013CE4B2029400240F4B87
:10AFC00001940095FFF792FD041E00D014E12900C2
:10AFD0007888FAF735FFDFE6486DFF1FC444FF1F8E
:10AFE0004C6AFF1F406AFF1F466BFF1F7C66FF1FF6
:10AFF0003C6CFF1FC244FF1FFFFF00004E6AFF1F93
:10B00000162406ABE41821003889FCF753FD011E15
:10B0100000D182E178882288AE4C45002C5BAE4D91
:10B02000013CE4B202947C89AC4B01940095FFF79B
:10B030005DFD041E00D0DFE029007888FAF70AFFE2
:10B04000AAE60025A44B1D803B00FE331B78A24AD4
:10B0500078880792AB4208D99E4B128806930699CE
:10B0600043005B5A013B9A4203DB0799FAF7FCFE67
:10B0700092E616246B00FB18059306ABE418059BBB
:10B0800021001889FCF716FD011E03D1059B012440
:10B090001E8973E77888924B2288069C09934300A7
:10B0A0001B5B904E013BDBB20293002300960193A1
:10B0B000099BFFF71BFD041E02D0059B1E895DE75F
:10B0C0007B88069A5B009B5A079A10883288121870
:10B0D000934202DC1B1A013B33807F4C02303288E2
:10B0E0000999001900F054FD2388328801359B1816
:10B0F0002380EDB2A8E70BAA3B7B798938890092BF
:10B100003A000D32FCF7EEFB00250590059B002B65
:10B1100004D10A24002D00D16EE060E0059B788800
:10B12000197AFCF7A9FB0100041E63D1694C6C4B32
:10B13000788806940993069B4400E45A694B063CC0
:10B14000E4B20BAE32880793029401910093059903
:10B15000099BFFF7CBFC041E4CD1079B5E491B8863
:10B160001A1D002D30D14A80059B5B4C5A8963190A
:10B170001A716B1C9BB2E318120A1A71162306A8E7
:10B1800032881B1879890598FCF708FDFF21AA1C55
:10B190002E1D03350B00059092B2B6B2ADB2002859
:10B1A00003D006ABDB8AD9B21B0AA218651911714C
:10B1B0002B714C4D301D2A884949201800F0E8FCBD
:10B1C0002B88F618B5B2A1E74988914207D17A8851
:10B1D00006995200525AEB18053A9A42C4DC3E4C8A
:10B1E0002800618800F0DCFB207021007888FAF7E5
:10B1F00045FED1E5002DF2D13E89BFE6162606AB0D
:10B20000F61831003889FCF755FC3D000400FF3585
:10B2100000282DD0037A9B060CD400227B89398923
:10B22000788800923A000C32FFF7E8FB041E10D039
:10B230003E8915E03088FFF741FB00281AD083686B
:10B24000002B17D02100122278889847041EE4D0E2
:10B25000EEE7AB78002B02D17888FAF71FFE0026C4
:10B26000AB78002B00D097E5002C00D194E585E663
:10B270000124DDE70E24DBE7162506ABED182900D7
:10B280003889FCF717FC041E47D0037A9B0611D4BB
:10B29000154A7B881188994203D01448814207D10E
:10B2A0001380134BF8261D780023D9B2A94221D36D
:10B2B0000924A1E72888FFF701FB00282FD0836825
:10B2C000002B2CD02100122278889847041EDFD052
:10B2D00092E7C0467C66FF1F4C6AFF1F4E6AFF1F45
:10B2E000466BFF1F3C6CFF1F406DFF1FFFFF000000
:10B2F0003C6DFF1F31005943546801336018615A97
:10B300000029D2D13C0008342100F82200F040FC92
:10B3100021007888FAF7CAFD3EE501246CE70E2487
:10B320006AE71D4B1A887B889A4231D07888FAF7F1
:10B33000C7FD31E5F823059851684343CD18C95A34
:10B3400000291FD03B7A012B0BD16C88AB88788801
:10B35000AA1D0094FFF752FB041E02D000233B728B
:10B360002E88F8220021280000F042FB00232B80C9
:10B37000059B0133DBB20593084B05991B78064A00
:10B380008B42D7D801235B421380002CCED0F5E549
:10B39000002634000596EFE7406DFF1F3C6DFF1F50
:10B3A00070B504000E001500FFF796FA031E08D1D1
:10B3B00031000548FFF790FA03001120002B02D05E
:10B3C0001C8000209D7070BDFFFF0000F8B50B4F82
:10B3D00006003B780D001400FF2B0ED00A2000F071
:10B3E00097FA011E09D0B123038000234680037120
:10B3F000C5800481387800F073FBF8BD1946FF1F43
:10B40000F7B50F0008A90600088809A90B240988C8
:10B41000002821D10234022B1ED1557813782D0239
:10B420001D432B008B4301937334002B14D1FB6815
:10B43000300019000093FFF74FFB019C85420BD0B1
:10B440002A0030000099FFF7ABFF041E04D12A0048
:10B4500030007989FFF7BAFF2000FEBDF0B50E7805
:10B4600085B003900AA805880120022E0DD14C68F2
:10B470002778647824023C43054FBC4205D10398E9
:10B48000DBB201960095FFF7BBFF05B0F0BDC046EB
:10B490000229000010B504000C4800F059F90C48CE
:10B4A000A16B00F055F90B48E16B00F051F90A4827
:10B4B000216C00F04DF9094B0948196800F048F972
:10B4C000084B1B68002B00D09847FEE7F6BC001124
:10B4D0000CBD00111BBD00112ABD001104ED00E0E0
:10B4E00039BD00114C6DFF1F002307B501A8019362
:10B4F000FFF7D0FF044A0548002110B5121A00F0EA
:10B5000077FAF8F759FAFEE7506DFF1F1C46FF1F48
:10B5100001B40248844601BC604700BF091B00001B
:10B5200001B40248844601BC604700BF6DBC000006
:10B5300001B40248844601BC604700BF3136FF1F9A
:10B5400001B40248844601BC604700BF093AFF1FAE
:10B5500001B40248844601BC604700BFA93BFF1FFD
:10B5600001B40248844601BC604700BF434D01005E
:10B5700001B40248844601BC604700BF2D3BFF1F59
:10B5800001B40248844601BC604700BF2951010054
:10B5900001B40248844601BC604700BFC53F0000BB
:10B5A00001B40248844601BC604700BF6932FF1FF6
:10B5B00001B40248844601BC604700BF311B000053
:10B5C00001B40248844601BC604700BF79180000FE
:10B5D00001B40248844601BC604700BF8B520100A1
:10B5E00001B40248844601BC604700BF9DA9000029
:10B5F00001B40248844601BC604700BF55490100C0
:10B6000001B40248844601BC604700BFC95C010028
:10B6100001B40248844601BC604700BFE117000046
:10B6200001B40248844601BC604700BFE548000001
:10B6300001B40248844601BC604700BF25260000D3
:10B6400001B40248844601BC604700BFE134FF1FDB
:10B6500001B40248844601BC604700BFF54E0100BA
:10B6600001B40248844601BC604700BF5118FF1F67
:10B6700001B40248844601BC604700BF75A90000C0
:10B6800001B40248844601BC604700BFB70E000009
:10B6900001B40248844601BC604700BFF94C010078
:10B6A00001B40248844601BC604700BFF539FF1F62
:10B6B00001B40248844601BC604700BF151BFF1F50
:10B6C00001B40248844601BC604700BF4135FF1FFA
:10B6D00001B40248844601BC604700BF3D4B0100F5
:10B6E00001B40248844601BC604700BFEDA50000DC
:10B6F00001B40248844601BC604700BF21460100F6
:10B7000001B40248844601BC604700BFF93CFF1FFA
:10B7100001B40248844601BC604700BFE92800002C
:10B7200001B40248844601BC604700BF9130FF1F4E
:10B7300001B40248844601BC604700BFB54C01001B
:10B7400001B40248844601BC604700BF8538FF1F32
:10B7500001B40248844601BC604700BFE53A0100DD
:10B7600001B40248844601BC604700BF5147010054
:10B7700001B40248844601BC604700BF055E00007A
:10B7800001B40248844601BC604700BF9137FF1FE7
:10B7900001B40248844601BC604700BF350E00007A
:10B7A00001B40248844601BC604700BF5D17000039
:10B7B00001B40248844601BC604700BF59520100F1
:10B7C00001B40248844601BC604700BFD13CFF1F62
:10B7D00001B40248844601BC604700BFC94A010069
:10B7E00001B40248844601BC604700BFA54F010078
:10B7F00001B40248844601BC604700BFADAE000002
:10B8000001B40248844601BC604700BFD949010029
:10B8100001B40248844601BC604700BF4D1F0000D0
:10B8200001B40248844601BC604700BFDD30FF1F01
:10B8300001B40248844601BC604700BF456B01006B
:10B8400001B40248844601BC604700BFD1A5000096
:10B8500001B40248844601BC604700BFC56D0100C9
:10B8600001B40248844601BC604700BF014C01009E
:10B8700001B40248844601BC604700BFDD520100AC
:10B8800001B40248844601BC604700BF1D4B010063
:10B8900001B40248844601BC604700BF3555000032
:10B8A00001B40248844601BC604700BF851F000008
:10B8B00001B40248844601BC604700BF691F000014
:10B8C00001B40248844601BC604700BF0189000002
:10B8D00001B40248844601BC604700BFB14E00007D
:10B8E00001B40248844601BC604700BF413AFF1FD3
:10B8F00001B40248844601BC604700BF0D520100FC
:10B9000001B40248844601BC604700BF45510100B4
:10B9100001B40248844601BC604700BF1D4D0100D0
:10B9200001B40248844601BC604700BF11470100D2
:10B9300001B40248844601BC604700BF6571010044
:10B9400001B40248844601BC604700BF3D180000B6
:10B9500001B40248844601BC604700BF8552010023
:10B9600001B40248844601BC604700BFD53BFF1FBD
:10B9700001B40248844601BC604700BFB537FF1FD1
:10B9800001B40248844601BC604700BFC5210000E5
:10B9900001B40248844601BC604700BF813AFF1FE2
:10B9A00001B40248844601BC604700BF090E000094
:10B9B00001B40248844601BC604700BF8132FF1FCA
:10B9C00001B40248844601BC604700BFB352010085
:10B9D00001B40248844601BC604700BF350E000038
:10B9E00001B40248844601BC604700BFC51D000089
:10B9F00001B40248844601BC604700BF154D0100F8
:10BA000001B40248844601BC604700BFC132FF1F39
:10BA100001B40248844601BC604700BF017F0000BA
:10BA200001B40248844601BC604700BFE53CFF1FEB
:10BA300001B40248844601BC604700BF090E000003
:10BA400001B40248844601BC604700BF7D18FF1F57
:10BA500001B40248844601BC604700BFF30E0000F9
:10BA600001B40248844601BC604700BFD91B0000F6
:10BA700001B40248844601BC604700BFCD4C0100C0
:10BA800001B40248844601BC604700BF5522000053
:10BA900001B40248844601BC604700BFC9A9000048
:10BAA00001B40248844601BC604700BF810E00001B
:10BAB00001B40248844601BC604700BF056A00002B
:10BAC00001B40248844601BC604700BF45500000F5
:10BAD00001B40248844601BC604700BF291C000035
:10BAE00001B40248844601BC604700BF594F0100C1
:10BAF00001B40248844601BC604700BF156B0100D9
:10BB000001B40248844601BC604700BFED4A010011
:10BB100001B40248844601BC604700BFA134FF1F46
:10BB200001B40248844601BC604700BF0933FF1FCF
:10BB300001B40248844601BC604700BF01240000F4
:10BB400001B40248844601BC604700BFA946010019
:10BB500001B40248844601BC604700BFC92600000A
:10BB600001B40248844601BC604700BF21240000A4
:10BB700001B40248844601BC604700BF3939FF1F49
:10BB800001B40248844601BC604700BF5125000053
:10BB900001B40248844601BC604700BFE94C010083
:10BBA00001B40248844601BC604700BF8D1200000A
:10BBB00001B40248844601BC604700BFC13AFF1F80
:10BBC0000002010302020303040305020602070246
:10BBD000080209030A030B030C020D020E030F03F4
:10BBE000100311031303140315001600813D001107
:10BBF000B53D0011000000000200000002BC001171
:10BC0000192A0F180A000000F1590000FD24000055
:10BC100041460100F17E0011059F0011597300118A
:10BC2000F57C0011615100112DAD0011194E00116C
:10BC3000793F0011A9400011000000001616000015
:10BC4000020000004CBC0011F4FFF3FFD2FC000026
:10BC5000654100110000000000000000547579618A
:10BC60000056302E38003030303100676974687506
:10BC7000622E636F6D2F70767678005448303500F1
:10BC80000200000094BC0011292A282A272A262A0B
:10BC9000252A242A0A180000E2040000710200008C
:10BCA00078EC0000744000001027000060F00000F5
:10BCB00006640000204E00000000000000000000AC
:10BCC0001F501D00023C020000011500080000008A
:10BCD000A30200003031323334353637383941422F
:10BCE00043444546005048592B36325858504C551D
:10BCF0005330353034005B48617264206661756C86
:10BD0000742068616E646C65725D0A004C5220207C
:10BD1000203D203078253038780A005043202020FC
:10BD20003D203078253038780A0050535220203D8D
:10BD3000203078253038780A0049435352203D207E
:10BD40003078253038780A0071550011C55500113A
:10BD5000000000000200000060BD00116F2A6E2A82
:10BD60001A18D880F060FFFFFFFFFFFFFFFFFFF30F
:10BD700003B59747D6F613F7D777E6F0A7F4740024
:10BD8000000001A0000000006410B71DC8206E3B39
:10BD9000AC30D9269041DC76F4516B6B5861B24DD2
:10BDA0003C7105502083B8ED44930FF0E8A3D6D63C
:10BDB0008CB361CBB0C2649BD4D2D38678E20AA0A4
:10BDC0001CF2BDBDFB349B5F8000008000100000B2
:10BDD000000000005B5F0011E57500117F5F00113E
:10BDE000ED79001103600011C37900117960001131
:10BDF00099790011CB600011617B00113361001152
:10BE0000617B0011656100111B7B001179600011DD
:10BE100051790011F1600011F97A00110000000061
:10BE200000000000D7610011F97A00113962001199
:10BE3000FD750011052A042A012A002A0229032877
:10BE40000128002801180018000000000000000070
:10BE50000000000000000087010102010201010250
:10BE600001020303040103010101010103030201B3
:10BE700003000D000E001000110013001401070153
:10BE800008010A010B011C011D0204020502070240
:10BE9000080219021A021C021D0301030203170003
:10BEA0000201000504000807000B0A001716001D18
:10BEB0001C010201010504010E0D011110011413F2
:10BEC000011716011A19020201020B0A020E0D02D5
:10BED0001110021413021716030504030807030BBD
:10BEE0000A030E0D0001020307090A0B0E0F1011C1
:10BEF00012141718191A1B1F2021220075A60011F1
:10BF000031A70011000000000200000046BE001131
:10BF1000000000005DB400110000000002000000FD
:04BF200044BE00110A
:020000041FFFDC
:1000000000000000DD3E001108BC001104BC00111E
:100010002863FF1F00000000000000000000000037
:1000200000000000000000000000000000000000D0
:1000300000000000000000000000000000000000C0
:1000400000000000000000000000000000000000B0
:1000500000000000000000000000000000000000A0
:100060000000000000000000000000000000000090
:100070000000000000000000000000000000000080
:100080000000000000000000000000000000000070
:100090000000000000000000000000000000000060
:1000A0000000000000000000000000000000000050
:1000B0000000000000000000000000000000000040
:1000C0000000000000000000000000000000000030
:1000D0000000000000000000000000000000000020
:1000E0000000000000000000000000000000000010
:1000F0000000000000000000000000000000000000
:1001000000000000000000000000000000000000EF
:1001100000000000000000000000000000000000DF
:1001200000000000000000000000000000000000CF
:1001300000000000000000000000000000000000BF
:1001400000000000000000000000000000000000AF
:10015000000000000000000000000000000000009F
:10016000000000000000000000000000000000008F
:10017000000000000000000000000000000000007F
:10018000000000000000000000000000000000006F
:100190000535FF1F5533FF1FC16601000000000039
:1001A000000000000000000000000000000000004F
:1001B000000000000000000000000000000000003F
:1001C000000000000000000000000000000000002F
:1001D000000000000000000000000000000000001F
:1001E000000000000000000000000000000000000F
:1001F00000000000000000000000000000000000FF
:1002000000000000000000000000000000000000EE
:1002100000000000000000000000000000000000DE
:1002200000000000000000000000000000000000CE
:1002300000000000000000000000000000000000BE
:1002400000000000000000000000000000000000AE
:10025000000000000000000000000000000000009E
:10026000000000000000000000000000000000008E
:10027000000000000000000000000000000000007E
:10028000000000000000000000000000000000006E
:10029000000000000000000000000000000000005E
:1002A000000000000000000000000000000000004E
:1002B000000000000000000000000000000000003E
:1002C000000000000000000000000000000000002E
:1002D000000000000000000000000000000000001E
:1002E000000000000000000000000000000000000E
:1002F00000000000000000000000000000000000FE
:1003000000000000000000000000000000000000ED
:1003100000000000000000000000000000000000DD
:1003200000000000000000000000000000000000CD
:1003300000000000000000000000000000000000BD
:1003400000000000000000000000000000000000AD
:10035000000000000000000000000000000000009D
:10036000000000000000000000000000000000008D
:10037000E9B40011000000000000000000000000CF
:10038000000000000000000000000000000000006D
:10039000000000000000000000000000000000005D
:1003A000000000000000000000000000951AFF1F80
:1003B000000000000000000000000000000000003D
:1003C000000000000000000000000000000000002D
:1003D000000000000000000000000000000000001D
:1003E000000000000000000000000000000000000D
:1003F00000000000000000000000000000000000FD
:081838005071FF1F4118FF1F52
:10184000024981F3088802F0E3FA00005071FF1F9B
:1018500010B502F01DFB072804D0122808D002287A
:1018600008D010BD044A0420136B01331363F8E75A
:101870000220F6E71420F4E72467FF1FF8B50700FD
:101880000C0026002500503630785135002804D150
:101890000300287058342370F8BD2978CA00481E08
:1018A0008141A3183800A25C5B68C9B2FFF7D0FF82
:1018B00000280DD12B78DA00A218013350602B706C
:1018C0003378044A013B3370136A01331362D8E75B
:1018D0000123DFE72467FF1F5C234343074910B55B
:1018E000C9180B0058331B78012B05D1FFF7C6FF31
:1018F000034A936A0133936210BDC0465867FF1FC5
:101900002467FF1F10B502F01BFA064A01211300DD
:1019100010CB4942D967044B136002F051FC200000
:1019200010BDC04600E100E01000100010B504003A
:1019300002F006FA024B1C6002F042FC10BDC046E9
:1019400000E100E010B5040002F0FAF94021094A74
:10195000200013688B43136002F022FB01F0B4FDFA
:101960000022054B01201A60044B04321A6002F079
:1019700007FBFEE71CF00040C4F00040C0F0004050
:10198000431E5A425341A022F0B5D2015B4213409C
:10199000154D164A40019B182A18127E8BB00191F2
:1019A000002A1BD01A000832D46F0022E6B206AF1C
:1019B000E4B294420EDC2818C369002B08D00199C8
:1019C00002AA117106AA049202AA167303A89847E4
:1019D0000BB0F0BD1978B9540132EAE71A7D1A78D4
:1019E00006AB01261A70E6E7E469FF1F00400040DD
:1019F000F0B5254B04004001C25C85B0002A2BD015
:101A00001A18117E002927D0917E002924D011793F
:101A1000022921D11689D788D168F51BADB22A1CBD
:101A2000102D00D9102292B2BE4217D118180123EE
:101A300003710023C269C38003819A4206D06846BD
:101A4000032103730171029301A890470820002C21
:101A500000D0192001F034FC05B0F0BD013C654216
:101A60006C41A0256442ED012C40084D1B186419FF
:101A7000074D0633013A92B2AA42EDD01888461CAF
:101A80001E80085C2070F5E7E469FF1F00400040FD
:101A9000FFFF00000F220E4B10B59868104002386F
:101AA0000A280BD802F01EF90D0A0B0A0A110A0ABD
:101AB0000A0A060002210020FFF762FF10BD012183
:101AC000F9E70020FFF794FFF8E7DB6FF6E7C04681
:101AD000004000400F220E4B10B5986810400238AD
:101AE0000A280BD802F0FEF80E0A0B0A0A120A0A9C
:101AF0000A0A060002210120FFF742FF10BD012162
:101B00000800F9E70120FFF773FFF7E7DB6FF5E760
:101B10000090004013B5334C2378072B3DD8324B4F
:101B20001A78324B002A39D18022196852020A43AE
:101B30001A60252001F084FF20232D4A11680B43F1
:101B4000802113606B460422C905086807331042E0
:101B500028D080210422C905C86810422ED08021D7
:101B60002020C905CA688243CA6014221A701A78F4
:101B7000002A2FD18021C905C86820320243CA60DB
:101B800014221A701A78002A28D11A4B1A7D22784A
:101B90005A601D221A705932DA6013BD1A6816494C
:101BA0000A40C5E7086802430A6014221A701A78CE
:101BB000002ACED01A78013AD2B2F7E7C8680243B9
:101BC000CA6014221A7019784A1ED2B21A700029FB
:101BD000F9D1C4E71A78013AD2B2C7E71A78013AC4
:101BE000D2B2CEE75445FF1F1C46FF1F3CF0004019
:101BF0004C45FF1F00200040FFFFFEFF564B70B515
:101C00001B68012B03D1554A936D0133936502F094
:101C1000EFF8534B534A1860534B544C1A6001234E
:101C2000534A1360534A13602378002B06D00622D0
:101C30005149524802F0F4FA00232370504A514BA4
:101C400010681B78C1B2002B0ED14F4CC0B2237864
:101C50005BB2002B4FDB237824785BB264B21B04A9
:101C600024021B191B1813600B1C50294ED950233A
:101C7000464A47491078DBB2FF2202284BD1086858
:101C8000444C454D267890432A78964254D9227880
:101C900024782E78023B5D10A31B6B435201D31AAC
:101CA00010335B111843086002F09AF8031F012BF0
:101CB00045D83A4B1B78002B06D0394B1B78002BAC
:101CC00002D0002002F03CFAA122364B9200997813
:101CD000354B4A431B689B18832292009B181B7844
:101CE000033B012B03D8AF20400002F059F801223A
:101CF0002E4BDA8270BD237824785BB264B2FF3356
:101D0000FF341B0424021B190138ABE7CAB2022AB4
:101D1000AED20223ACE70868254C264D26789043C6
:101D20002A78964208D9227824782D78023B5B10D5
:101D3000641B63435201B2E72378DBB2B2E70228A7
:101D4000D5D11D4B1B78013B022B03D91B4B1B78B4
:101D5000022BCCD16C20C8E79809FF1FFC0FFF1F96
:101D60005C66FF1FFF3F0000141003406066FF1F0A
:101D70000C10034000100340D50BFF1F7211FF1F12
:101D8000B40003408C09FF1F680AFF1F490AFF1FA8
:101D900094000340460AFF1F470AFF1FF908FF1F70
:101DA0002209FF1F300DFF1F3409FF1FBC0BFF1F4F
:101DB000440AFF1F450AFF1F1C09FF1F2309FF1FBD
:101DC00010B502F0E5F90022014B1A8010BDC046A3
:101DD0005866FF1F10B502F07BF9A121054A890062
:101DE0009478054A61431268044B5218528C1A8049
:101DF00010BDC046300DFF1F3409FF1F5866FF1F7E
:101E000010B50D4B0D4A9978A1239B004B431268E6
:101E1000D218531DD97F0A4B1B88994209D2441C02
:101E200007D0C82805D0D2695B1A5A43054B5343E3
:101E3000C01801F095FF10BD300DFF1F3409FF1FC2
:101E40005866FF1F7102000070B5244D2B68002BEF
:101E500028D001F05DFF2B68D8402B680400002BD0
:101E600027D001F095FF2B68D8401D4B1D4A99786B
:101E7000A1239B004B431268D118D25C91239B0095
:101E8000002A20D0CA580132CA50174B17491B6884
:101E90000868834214D3D23B181A012A1AD0144B73
:101EA000186070BD01F034FF124B196802F050F950
:101EB000D3E701F06DFF0F4B196802F049F9D4E741
:101EC0000D495B18E8E7CA500C4B1B68DB68E41847
:101ED000201AE4E7F530FF30E1E7C0461C08FF1F99
:101EE000300DFF1F3409FF1F9C09FF1F5C66FF1F99
:101EF000A009FF1F1808FF1F2DFF3F006466FF1F8A
:101F000070B504000D00282916D10300A433C2883F
:101F10001B889B1A0B4A9BB293420DD906006A3666
:101F200005223100653001F053FF002804D1310053
:101F3000200002F09DF870BD2900200002F018F981
:101F4000F9E7C046FE7F0000F8B50400012002F06A
:101F50006FF802F075F8174A174910600968030016
:101F60001648174E01601748776805680020AF4291
:101F700001D27068281A144D091928601348C162EB
:101F8000A421446A49032143416211490978002987
:101F900005D010490978022902D10F3B1360F8BD22
:101FA000012901D1083BF9E7032901D1053BF5E7F8
:101FB000033BF3E7E408FF1F28F00040340AFF1F4B
:101FC00028100040180AFF1F1C0AFF1F00F00040E5
:101FD0001C09FF1F4A0AFF1F70B580241025E40565
:101FE000A3682B43A36001F03BFFA368AB43A3604E
:101FF00070BD0000F7B5160080221C001023D2052A
:102000000191916805000B43936000225A4BD73031
:102010001A6001F015FF9D232A002F009B00EB584A
:10202000CA3201210092FC37002B01D00021009A16
:10203000386801F0E5FF2900009BCB311A784F4B3F
:10204000D3351A604B780A781B0213438A7812043E
:102050001A43CB781B061343494A1BBA13604B79CA
:102060000A791B0213438A7912041A43CB7931008F
:102070001B061343434A1BBA13606B782A781B0272
:102080001343AA7812041A43EB781B0613433E4A03
:102090001BBA1360019A330213433C4A13603C4B52
:1020A00022001B1B9C4603293DDCB3089A00130049
:1020B0005142B21A032A46D1354AE018511A8278A1
:1020C0004078120400020243E05C043302430A60D9
:1020D0000022FF2B4BDDF0222E4B12011A600F2243
:1020E0002D4B1A602D4A1368002BFCD00023224A86
:1020F00027491360091B321D0B191B68043A180A83
:1021000023706070180C1B0EA070E3700434002A5A
:10211000F2DC802210213B68D20501333B609368DA
:102120008B439360F7BD6346D578981893782D0656
:102130001B042B43157804392B43557804322D02A8
:102140002B430360AFE7022A0AD1114AE05C511A1F
:10215000E2185278120202430A6004339BB2B7E7D6
:10216000012AB5D10A4A521AE15C1160F5E7084923
:1021700059180A600433ACE7000004403C000440F6
:102180003800044034000440300004400C00044097
:102190000001044004000440100004401400044006
:1021A000F7B5150080221C001023D205009191681C
:1021B00007000B4393600023654AD730136001F09A
:1021C0003FFE9D233E009B00F9583B00CA3632007B
:1021D000FC33002900D07FE0586801F011FF39007E
:1021E00032785C4BCB311A604B780A781B02134370
:1021F0008A78AC4612041A43CB78281D1B06134379
:10220000554A1BBA13604B790A791B0213438A792A
:1022100012041A43CB791B061343504A1BBA1360AE
:102220004B7A0A7A1B0213438A7A12041A43CB7A36
:1022300021001B0613434A4A1BBA1360009A2B0263
:102240001343484A13602200474B1B1B0093009B1B
:10225000CE785B1801938B7836061B0433430E78D7
:10226000043833434E78043136023343019E3360E1
:102270000328ECDC0321A808431C9B0029408000B4
:1022800003292BD13849E5185E18A9786D78E35CED
:1022900009042D022943194331600300083300214A
:1022A000FF2B2DDD314B324919600F21314B196065
:1022B000012327490B60304B19680029FCD0062107
:1022C0001B680B40042B20D080220020D20593688D
:1022D0000A318B439360FEBD01217DE7022908D1BD
:1022E00021495D18E1184978E35C09021943296026
:1022F000D3E70129D3D11C495918E35C0B60CCE723
:102300001948181801600433CAE7002310490B600C
:102310006346002B0CDC3B00FC335A681021013271
:102320005A608022D205936801208B439360D2E7E4
:10233000009B9B181B68190A13705170190C1B0E17
:10234000D37004235B4291709C440432E0E7C046A2
:10235000000004403C0004403800044034000440C5
:10236000300004400C00044000010440040004401C
:10237000080F0000100004401400044070B5061E51
:1023800019D00222614B9B799343012B13D1604BEF
:102390001A78FF2A0FD15A78FF2A0CD19A78FF2A8F
:1023A00009D1DA78FF2A06D11A79FF2A03D15B799D
:1023B000FF2B00D1A7E0574B0C201A78012A08D038
:1023C0000022554D1A702B781A00093A042A01D8B8
:1023D000212070BD5A1F012AFAD94C4CA07B042839
:1023E00000D990E0A279032A00D98CE0821E012A4C
:1023F00003D862881F2A00D885E0002E61D0012E04
:1024000000D080E0A288012AE2D0002B0AD1013856
:10241000032803D801F066FC151D19151F202E7026
:1024200001F04EFD2B785A1E032A16D800253B4B8F
:102430001D602823237501F0ABFDA8422ED0A58096
:10244000C6E7022320202B70EAE7042322202B700A
:10245000E6E7032321202B70E2E7073B012BB7D8E7
:102460002F4B1B68DB6A9B06B2D52E4B1A78002ACD
:10247000AED1A27B911E012901D9002AA8D1022246
:1024800080211A702823284D89012878237501F0AE
:102490006FFD80212878890101F00AFE0123A380C5
:1024A000224B1B78002B0AD0FA228021204B92006D
:1024B0001B8809025A431C4B187801F091FE00203A
:1024C00087E701F03DFC2B78A680073B012B06D95E
:1024D00018482E7001F00CFD1E2001F0F1FC114B8C
:1024E000114C1A78002A06D0802100222078890118
:1024F0001A7001F03DFD01F063FE80212078090291
:1025000001F036FDDBE7122063E7C046A60BFF1F94
:102510006B09FF1F1A09FF1F1C09FF1F4809FF1F36
:102520006466FF1F2309FF1F1B09FF1F2109FF1FEF
:102530002C09FF1F0010004010B5002901D001F048
:10254000F7FD10BDF7B5604B01919978A1239B0071
:102550004B435E4A060014681022E418D6235B0041
:10256000E0583623FF33E35C00279343222B41D10D
:10257000574B0F3A1A600760012501F049FD019B96
:102580001880E8235B00E35C002B01D0B34258DDE8
:102590000023504FFB70AD33FF33E3581A68002A15
:1025A00003D09B88DB439B071DD03823FF33E35CBC
:1025B000002B18D09B235B00E35C002B13D1D1339D
:1025C000FF33E35CB3420EDAA4235B00E15AE01868
:1025D000090A023101F03CFC23000122FE33013ED6
:1025E00001351A87FA70E8235B00E35C002B2AD0E0
:1025F000A8B2FEBD03683D00002BBED08188043028
:10260000090A023101F024FCD6235B00E3581F6065
:10261000B2E72300B133BA00FF33985801378188FD
:102620000430090A023101F013FCE8235B00E35C8B
:10263000BB42EEDCE822F61AED1800235200A35448
:10264000A6E70027F1E7200001F08AFD00281FD04F
:10265000002E1DDD7319882647190193B60020004E
:1026600001F0A6FD5A3080002018406801358188AD
:102670000430090A023101F0EBFB200001F080FB7D
:10268000A3590133A351BD4202D0019B9D42E6D123
:10269000114BE35C002BABD095239B00E35C002B3C
:1026A000A6D00E4BE15A0029A2D00D4AA35C994254
:1026B00002D90133A3549BE700231A212000A3541D
:1026C00001F056FB94E7C046300DFF1F3409FF1F91
:1026D00000140340E010FF1F5A02000072020000C5
:1026E0005E020000F8B51D4B1D4F1A78002A10D16C
:1026F000BA7B002A02D101321A7003E0032AFAD011
:10270000022AF8D001F044FC00220120154B1A7077
:10271000F8BD154B154D1C68154B9E7801232B7089
:102720002878C0B200F0DEFCBB7B002B0BD101F09F
:102730007FFDA1239B007343E41883239B00E418CF
:1027400023782B70E4E7032B02D101F041FCF0E782
:102750000020022BDCD101F0E3FCEAE71C09FF1F9B
:10276000A60BFF1F2309FF1F3409FF1F490AFF1F84
:10277000300DFF1FF0B587B00EAD2F780FAD2D785F
:102780000593AC46634614000E4D0CAA12782E78C1
:1027900003930D9B009201932200059B029701F089
:1027A000B7FB2E70012C01D0042C08D180220649E1
:1027B0008B889343054A1278D20113438B8007B06C
:1027C000F0BDC0461C09FF1F6C11FF1F7809FF1FD9
:1027D0000B001B3B70B504003020E02B0DD813001C
:1027E000E025493BFF3B9BB2ED00AB4205D8034BD4
:1027F000200019825A8201F06BFB70BD8410FF1F0C
:1028000010B501F0F5FA054B00205B68052B04D9E3
:10281000034A5268D20200D4980810BD001000404C
:10282000FCE100E070B501F08BFA0D4B1B68FC3346
:10283000DC691D6AFFF7E4FF6419844204D2094B86
:1028400001241B68002B07D004220024064B1A70B9
:10285000064A93690133936101F0B2FC200070BD18
:102860006466FF1F9809FF1F2309FF1FFC0FFF1F4E
:1028700070B50C4D2B68FC335C6A01F061FAFFF710
:10288000BFFF2B680025FC339B6AE318834204D208
:10289000054B1B68AB4200D1051B01F091FC2800E1
:1028A00070BDC0466466FF1F9809FF1FD722044B06
:1028B00092009B5810B5002B00D0984710BDC04621
:1028C0000000FF1FF0B587B001F096F9FFF7EEFFAB
:1028D000CA4BCB4C04931B78022B45D1C94B1B68C8
:1028E000186A01F0A5FBC84BC84A1A60C84BC94A10
:1028F0001A60A022C84B52001A60049B187801F09D
:102900007FFCC649C64801F0A3FBC649C64801F092
:102910009FFB1022C54BFF201A60802252031A60D1
:10292000802292031A60802212041A6001F008FCCF
:10293000012001F0A5FAFA20400001F041FB5820E7
:1029400001F02EFABA4801F00BFB012001F080FCE7
:10295000072001F0EDFA2268B64B1A4084235B0091
:102960001343236007B0F0BD01F0DAFAB24E0290D3
:10297000322001F05DFB33681B0629D43C2001F0B6
:1029800057FB0F2001F054FB9C4B1B78012B00D10F
:102990001EE180223368A94D134200D0A7E02B68C6
:1029A000032013432B6001F043FB01F0B9FA029BB3
:1029B0000299C31A5A1E814200D81A00A04B1A600D
:1029C000904B19681E2353439E4A9B18CB618AE79C
:1029D00001F0A6FA80239C4ADB02116803900B43A6
:1029E00013602268934B994F1A40282313432360A6
:1029F000032001F01DFB03203D6801F019FB3B683B
:102A00000320DB03DB0B009301F012FB3B68ED03BB
:102A1000DB03ED0BDB0B8E4A0193AB18C22B30D8D6
:102A2000009B9B18C22B2CD8019B9B18C22B28D82B
:102A3000009B2A009D4200D21A00009B9D4200D9B3
:102A40001D00019B934200D21300019A954200D9C8
:102A500015005B1B122B14D80C22336814209343EF
:102A6000336033687B4A1340336001F0E1FA082198
:102A70003B682268DB038A432260774ADB0B1360E2
:102A80007FE7032001F0D4FA3B68DB03DB0B0593FF
:102A900001F046FA039B0399C21A531E814200D8E3
:102AA00013006E4A93421BD9FF23356869492D0AEA
:102AB0001D4032686B1C1B060A401B0C134333601D
:102AC0000C23326800209A43083B1343336001F023
:102AD0008FFB6348634BA840984206DCFEF732FF49
:102AE000019B009D0093059B95E75F48F6E7002357
:102AF0005E4F554A3B6080231168DB020B43136035
:102B000080222B68032013432B6001F091FA3B686D
:102B1000052601333B6080232A685B0213432B6048
:102B20002268444B03201A40514B1343236001F0A9
:102B30007FFA0821454B1A682368D2038B43236030
:102B4000454B023900931B68D20B4B439A420CD879
:102B50009B1A3B2B0BD8236846490B4023602B68FC
:102B60000B402B60444B1A601FE7D31AF1E7013E7C
:102B7000F6B2002ED4D123683E4A134023602B685E
:102B800013402B603B68042B07D9BFF34F8F3B4B9F
:102B90003B4ADA60BFF34F8FFEE780222B680320A9
:102BA00093432B6001F044FA2268224B03201A4021
:102BB00028231343236001F03BFA244B009A1B683F
:102BC000DB03DB0B1360082223689343236097E742
:102BD00007222C4D2B681340012B02D1002001F05D
:102BE0000FFBAB68284A02201340AB6001F020FACB
:102BF0008023AA685B001343AB60D6E64A0AFF1F36
:102C00005CF000406466FF1F000003400180063D49
:102C1000BC00034034080000A4000340710200001F
:102C200014100040FFFF3F002810004000E100E0CA
:102C30003075000000FEFEFFC4F0004044F000408C
:102C40004C66FF1F7206000040F0004064F0004038
:102C500091FCFFFFFF00FFFF5466FF1FE30C000025
:102C6000E88000005F361E0060361E00B844FF1F7B
:102C700028000100FFFFFEFF5066FF1F00ED00E08F
:102C80000400FA053CF00040FFFEFFFF694E336888
:102C900088331B6883F3088801F0B2F800F014FC55
:102CA000654B664A1B68934207D0002001F0A0FAEA
:102CB0000221634A13688B431360FFF703FE614BE5
:102CC000614C1878C0B201F083FA0023A36002338C
:102CD000A3605E4B0120236001F0AAF90323A360E7
:102CE00001F01EF9040001F083F8050001F018F965
:102CF000574B186001F02CF9564B1968621A531E95
:102D0000A14200D213008022D203934201D39B023E
:102D10009B0A3268D16AC90700D478E04E491C0C7E
:102D200009689BB24C4359432402090A64180327DB
:102D30004A49FC3293680A6849489B1A494A4A4EF4
:102D400012684A499B18414A34609A183B400193E3
:102D5000036892089C46019B0A6063440360042B4D
:102D600003D901323B400A6003600B684049E41814
:102D7000200001F0EDF93F4F3D493B68C3183B602F
:102D80002000019300F0D4FF3B4C2068081838491C
:102D90002060884205D9019B01333B6000F0C8FFE9
:102DA000216001F04DFA354B1B78002B0ED001F05D
:102DB0001FF83168324B4A1B1B6812189A4233D2F3
:102DC000591A4919091A2F4801F042F92E4C237A51
:102DD000002B0FD001F00CF83168E3684A1B121881
:102DE000934224D9591A4919091A284801F030F98F
:102DF00000232372264B83F3088801F0D1F90220C7
:102E000001F05EF8002001F0F3F901F031F8DC0187
:102E100099000234641A5900641A09214B43803323
:102E2000CB40A408E41882E7FA218900CBE71949CE
:102E3000DBE7C0466466FF1F0C0AFF1FB641210393
:102E400010000040490AFF1F14100040C409000090
:102E5000100AFF1F340AFF1F380AFF1F200AFF1F36
:102E6000280AFF1F1C0AFF1F4866FF1F240AFF1FB6
:102E7000710200006008FF1F2C0AFF1F1C09FF1FC2
:102E8000E408FF1F00100040740BFF1F3C100040BF
:102E900000000020DC050000A022054B92009B589A
:102EA00010B5002B01D0984710BD01F019F9FBE7D0
:102EB0000000FF1FA122054B92009B5810B5002B6C
:102EC00001D0984710BD01F00BF9FBE70000FF1F90
:102ED000A222054B92009B5810B5002B01D09847B9
:102EE00010BD01F0FDF8FBE70000FF1FA322054B1A
:102EF00092009B5810B5002B01D0984710BD01F0EF
:102F0000EFF8FBE70000FF1FA422054B92009B583F
:102F100010B5002B01D0984710BD01F0E1F8FBE798
:102F20000000FF1F70B500F063FF514B18600420D4
:102F300000F0C6FF00F074FF0400C30702D400F0E5
:102F4000B7FF70BD00224B4B1A604B4B187801380D
:102F500004282CD800F0C6FE03231B1F27002000E6
:102F600001F096F80128ECD0444C2378042B71D161
:102F700001F0CEF8002806D000F0D2FE582000F074
:102F80000FFF02232370032000F09AFFD9E72000EF
:102F900000F04EFFE6E7200001F00AF8E2E720002B
:102FA00001F06EF8DEE7200001F032F9DAE700F018
:102FB00017FF0500012808D1314B1B78053B012B79
:102FC00003D82000FFF768FFCEE72C4B1B78022BBD
:102FD00001D0052B20D1022D28D12A4B9B7BAB435E
:102FE0001CD12000FFF766FF254B18780128BBD1C4
:102FF0006405B9D4234925224B7B034205D1233AEA
:1030000013405A42534126331A000B7D9342ABD9E9
:10301000322000F065FFA7E7022D07D1184B1B787F
:10302000052B11D12000FFF753FFDDE7012D0BD158
:10303000012B03D12000FFF759FF95E7062B03D1A1
:103040002000FFF761FF8FE7200001F049F8022D13
:103050008AD1C9E7032B04D10B4B987C00F070FF99
:1030600091E7072B8FD1094B987B01F041F88AE754
:103070009C09FF1F9809FF1F9009FF1F2309FF1FCD
:103080001C09FF1FA60BFF1FBC0BFF1FD40BFF1F4C
:10309000FA210A4B0A4A49001A640A4A5A500A4A53
:1030A00004395A50094A08319A64094A5A50094A5F
:1030B0005C315A50084ADA667047C0460000FF1F6C
:1030C0007527FF1F7128FF1F2528FF1F7D23FF1F66
:1030D000E526FF1F011EFF1FD51DFF1F10B500F0C5
:1030E000E9FD10BD8023F7B59C46264B264F019382
:1030F0002649274A274D284C284B02281AD16046DA
:1031000038600868264E3040802636033043086019
:1031100001990978002909D11660224A2A60224AB9
:103120002260E02219689143A03A1BE08021C90285
:103130001160F2E766463E600F68194E3E408027F8
:10314000FF023E430E600199097800290DD11760F6
:1031500001280ED1154A2A60154A2260E02219681A
:103160009143C03A0A431A60F7BD80218902116079
:10317000EEE7E0210F4A02432A600F4A22601A68F4
:103180008A43F0E74B0AFF1FE0000340D8000340EA
:103190009000034000000340500003404000034003
:1031A000FFFFE3FF0280063D804508220180063DC7
:1031B000806608220080069880550822F8B51E4BCC
:1031C00080261A68002014003440324232D11A6836
:1031D0001A4F32431A6001223B68063093433B602A
:1031E00000F026FF0122164D2B681E432E603B681F
:1031F0000A2613433B608027BF00124B1B683B42EB
:1032000011D1013EF6B2FF2E09D17E220E4B1C6871
:103210002B68E40B1440934323432B6005E0082004
:1032200000F006FFE9E7002EEFD180222B6860084E
:1032300093432B60F8BDC046C4F000405CF00040F2
:1032400018F0004068F0004060F0004010B500F059
:10325000B7FD01215820034A00F052FEFFF7AEFFF0
:1032600010BDC046600AFF1F10B578220021034838
:1032700000F086FF00F0F4FE002010BD6C69FF1F17
:1032800070B5040000F05CFD00230C200B4A010027
:1032900059438D18515C00290DD0A14208D101235A
:1032A00000246B7000F0A4FE00F08AFF200070BDC7
:1032B00001330A2BEBD11224F6E7C0466C69FF1FDD
:1032C00070B5040000F03CFD002319001D000D4AFC
:1032D0001078002806D0A0420CD1557001310C3274
:1032E0000A29F5D1002B0AD100F0BAFE00F068FFE0
:1032F000002070BD5078461EB0411B18EEE700F06C
:1033000077FEF3E76C69FF1FF7B504000C2000237C
:1033100084460E4D019267465F43E85D7E19A042E8
:1033200012D000280BD10A4B9C4662461B7808330A
:103330001370019B70707C557160B360FEBD0133EA
:103340000A2BE8D10320F9E70720F7E76C69FF1F94
:103350006869FF1F8021F8B5464BC9051B68C12469
:103360008B60454BFF261A68012313434B61434B87
:10337000A4001A68424B40201A60424B1A68424B24
:103380001A60424B1A59B2431A51C52292009D58F5
:10339000B5432843802598509F583D48ED0107408C
:1033A0003D439D509D5880272D022D0A2943995059
:1033B00080211A59090202400A431A5104341A5949
:1033C000344D3F042A403A4380271A511A593F0688
:1033D0001202120A3A431A5108341A5902400A4397
:1033E0001A51C32292009D58B5432C0080252C43CE
:1033F0009C509D582C0004400C439C509D58254CDB
:1034000025408024240425439D509C588025240277
:10341000240A3C439C50C424A4001A59B2432A43B2
:103420001A511A591202120A17431F5108341A5915
:10343000B24315431D5100251A5902400A431A513F
:1034400004341A59024011431951134C134B1B7881
:10345000DB08AB4201DC0020F8BD2378002B06D04E
:10346000A368002B00D0984701350C34EEE71220FA
:10347000F2E7C0465045FF1F4C45FF1FB0F000402B
:103480006469FF1FB4F000406069FF1F00E100E0C5
:10349000FF00FFFFFFFF00FF6C69FF1F6869FF1F50
:1034A000030010B51F2809D8072200201340072465
:1034B00004490A78A24313430B7010BD0023062071
:1034C000F5E7C0466869FF1F034A044913680020F6
:1034D0000B4013607047C0461CF00040FFFFC1FF67
:1034E000054B06491B780A6805485B0702401B0B21
:1034F000134300200B6070476869FF1F1CF00040F9
:10350000FFFFC1FF70B50C25FFF7EAFF0A4B1C78DF
:103510000A4BE4086543ED18002C01D1200070BD72
:103520002B78002B06D06B68002B00D09847013C0D
:103530000C3DF1E71220F2E76869FF1F6069FF1F89
:1035400007B50422074801A900F034F9019B0133B3
:1035500005D18023044ADB0411680B43136000206B
:103560000EBDC0461C18001114F00040F0B5050057
:103570002026184B87B00493049B002B03D1112401
:10358000200007B0F0BD002102220B000191009144
:10359000052000F00DFC02230F490A681A42FCD1F5
:1035A0000596059C631E0593002CFAD10B4A1368FF
:1035B000002BFCDA0F276F440121380000F070FD6A
:1035C0003B782B42DCD0052000F032FD049B013B10
:1035D0000493D1E7FFFFFF0790C8004000C80040F8
:1035E00007B500F0ADFB80220821D205936A019156
:1035F000002B01D10739916202210C4A1160019917
:10360000481E01900029FAD1033111600531019162
:103610000199481E01900029FAD11160002B02D1B6
:103620008022D205936200F0CBFD07BD00C00040B0
:10363000F0B52D4C89B02378002B4FD1FEF762F9FD
:1036400002232A4F03903A681A42FCD120230693A2
:10365000069B5A1E0692002BFAD1254E3368002B8A
:10366000FCDA0120FFF782FF011E02D0112009B011
:10367000F0BD030003220190009005AD9F2000F0F3
:1036800097FB0321280000F00BFD02233A681A4241
:10369000FCD120230793079B5A1E0792002BFAD1D7
:1036A0003368002BFCDA0120FFF760FF0028DDD132
:1036B0000398FEF73BF9AA786B7811041B020B43C1
:1036C00029780B4363601300113B0A49052B07D887
:1036D00001239340A3600B60012323700020C6E701
:1036E00080231B03F6E7C0463845FF1F90C8004003
:1036F00000C800409808FF1F1E4B30B55A68187864
:103700001D4B85B0D31859424B4101210093002332
:1037100000F0D6FC194B1A4A02259A6300221A655A
:1037200010325A658022C4219D65164B1648D2027C
:10373000DA6789004258154B80241A4080231B0405
:1037400013434350642341200393E40500F078F9C8
:10375000402000F075F96562039D6B1E0393002DF8
:10376000FAD103236362FFF73BFFA562FFF760FF17
:1037700005B030BD4445FF1F95FFFEF700C800406F
:10378000050001FF04E100E000E100E0FFFF00FFB1
:1037900010B5064B18705960FFF7AEFF00211320DB
:1037A000034AFFF7B1FD002010BDC0464445FF1F8E
:1037B000F936FF1FF0B5040085B003920291FEF7C1
:1037C000A1F8882263035B0B52051A438023DB05B3
:1037D0009D6A8023274F0092BA68002601901B0340
:1037E0009A420CD9F82326001B041E401C4206D026
:1037F0008022214B52025E6219680A431A60002D32
:103800000BD100F09DFA02221C4B1A608023DB05CD
:103810005A62013A9A6200F0D3FC0023039A934261
:1038200020D1002D0AD100F08BFA144B03221D6029
:103830008023DB055A629D6200F0C2FC8023BA68D7
:103840001B039A4208D9002E06D000220A4B0C49CD
:103850005A621A680A401A600198FEF767F8002059
:1038600005B0F0BD009A0299D2181278CA540133FB
:10387000D4E7C0463845FF1F00C8004000C00040E4
:10388000FFFFFEFFF0B587B0029103920400FEF740
:1038900039F8019000F054FA802302250122234ECA
:1038A000DB0535605D629A6200F08AFC204F3B6860
:1038B0002B42FCD120230493049B5A1E0492002B1C
:1038C000FAD11C4D2B68002BFCDA0120FFF74EFECD
:1038D000002802D0112007B0F0BD2000039A029901
:1038E00000F0DEFA022304003A681A42FCD12023D9
:1038F0000593059B5A1E0592002BFAD12B68002BCD
:10390000FCDA0120FFF732FE051EE3D100F018FAC1
:1039100080230322DB0535605A629D6200F050FC73
:103920000198FEF703F8E0B2D5E7C04600C00040BA
:1039300090C8004000C80040F0B5802687B0040061
:10394000FDF7E0FFF605B36A02250393029000F04D
:10395000F7F90123244F3D607562B36200F030FC3B
:10396000224E33682B42FCD120230493049B5A1E21
:103970000492002BFAD11E4D2B68002BFCDA01209B
:10398000FFF7F4FD002802D0112007B0F0BD2000A1
:1039900000F026FB0223019032681A42FCD120235A
:1039A0000593059B5A1E0592002BFAD12B68002B1C
:1039B000FCDA0320FFF7DAFD041EE5D100F0C0F9C0
:1039C00080230322DB053C605A629C6200F0F8FB16
:1039D000039B002B01D1FFF703FE0298FDF7A6FF22
:1039E0006B461879D1E7C04600C0004090C800403F
:1039F00000C8004007B5000201910422000A01A995
:103A0000FFF740FF0EBD000073B5050005240B4A0B
:103A1000A3005B429B1819686B46DE1D300000F066
:103A2000FFFA022804D133782B55013CEFD276BD42
:103A3000052CFCD00128FAD10230F8E71409001156
:103A40001F2807D8012380228340D20591680B43A9
:103A5000936070473F2808D8012380222038834094
:103A6000D20551690B435361F3E75F28F1D8012375
:103A7000802240388340D205116A0B431362E8E785
:103A80001F2807D8012280218240C9058B689343F3
:103A90008B6070473F2808D801228021203882405F
:103AA000C9054B6993434B61F3E75F28F1D80122C5
:103AB000802140388240C9050B6A93430B62E8E7D6
:103AC0001F2810D880230200DB05153A1968012A47
:103AD00006D820229143196019680A431A6070477A
:103AE00001228240F6E73F2811D880230200DB053F
:103AF000353AD968032A06D810229143D960D9688B
:103B00000A43DA60EBE7012220388240F5E75F28BC
:103B1000E5D842238022181A413B8340D205516ADE
:103B200099435162516A0B435362D8E710B50400C0
:103B3000012813D1A022184992050B685B015B098B
:103B400013430B60154B164A19681140154A0A4376
:103B50001A60402219680A431A6010BD0028FCD17F
:103B600001000A2000F0CCFA21000B2000F0C8FA76
:103B7000C0220A4B920019680A4340211A601A6851
:103B80008A431A60B022044912060B685B015B0984
:103B900013430B60E1E7C04614F000401CF0004006
:103BA0007F00FEFF80FD010072B6074A13680133F3
:103BB00013600422054B1A600023054A136080221B
:103BC000D2055360FEE7C0467808FF1FC0F00040F2
:103BD000C4F00040044B054A1A60054B1A600022ED
:103BE000044B1A607047C046140AFF1F841E000071
:103BF000380AFF1FC4F000400023034A1360034A41
:103C00001360034A1360704754F0004040F10040D5
:103C100044F10040002310B5184C8AB00093019382
:103C20002378012B27D06946012000F091F8002865
:103C300017D1009B12490293019B06AA0393114BD3
:103C400002A81B680493104B1B68059300F008F949
:103C500010220E4906A800F0BBF8002804D1FF236B
:103C6000237000200AB010BD0123094A074902A8A9
:103C7000237000F0F5F80120F4E7C0466866FF1FE6
:103C800010290011082900110C2900112029001108
:103C90006C66FF1F13B501246946012000F058F837
:103CA000034B00940193FFF7B5FF200016BDC046FB
:103CB000BB0B000010B5FFF79FFFFFF7EBFF0028DD
:103CC00002D0024B984710BDFEE7C046E1A20000BB
:103CD00002B4714649084900095649008E4402BCA5
:103CE0007047C04602B4714649084900095C490062
:103CF0008E4402BC7047C04603B471464908400078
:103D00004900095A49008E4403BC70470000000076
:103D100001B40248844601BC604700BFE90B0100C2
:103D200001B40248844601BC604700BF6DF6000044
:103D300001B40248844601BC604700BF090E000080
:103D400001B40248844601BC604700BF75A9000069
:103D500001B40248844601BC604700BFE1AC0000EA
:103D600001B40248844601BC604700BF89370100A6
:103D700001B40248844601BC604700BF53B900004B
:103D800001B40248844601BC604700BF5976010077
:103D900001B40248844601BC604700BF6D0B0100BE
:103DA00001B40248844601BC604700BF791201009B
:103DB00001B40248844601BC604700BF496D010060
:103DC00001B40248844601BC604700BFED680100B1
:103DD00001B40248844601BC604700BFCD4C0100DD
:103DE00001B40248844601BC604700BFDD0C0100FD
:103DF00001B40248844601BC604700BFC95C0100B1
:103E000001B40248844601BC604700BFC9A9000054
:103E100001B40248844601BC604700BFF5B40011FC
:103E200001B40248844601BC604700BFBD0B0100DD
:103E300001B40248844601BC604700BF0934010058
:103E400001B40248844601BC604700BF89440000B9
:103E500001B40248844601BC604700BFC11501009F
:103E600001B40248844601BC604700BFDD3F00004A
:103E700001B40248844601BC604700BF855201007E
:103E800001B40248844601BC604700BF69110100CB
:103E900001B40248844601BC604700BFE927000026
:103EA00001B40248844601BC604700BF957301001D
:103EB00001B40248844601BC604700BFDD0A01002E
:103EC00001B40248844601BC604700BF19070100E5
:103ED00001B40248844601BC604700BF116E000077
:103EE00001B40248844601BC604700BF613701004D
:103EF00001B40248844601BC604700BFC1A5000070
:103F000001B40248844601BC604700BF016701005C
:103F100001B40248844601BC604700BF9D6A0000AE
:103F200001B40248844601BC604700BF156B010024
:103F300001B40248844601BC604700BFF90D01008E
:103F400001B40248844601BC604700BF4DF900003F
:103F500001B40248844601BC604700BFC16601004D
:103F600001B40248844601BC604700BF8D110100C6
:103F700001B40248844601BC604700BFB35201004F
:103F800001B40248844601BC604700BFA1AF0000F5
:103F900001B40248844601BC604700BFA9D80000B4
:103FA00001B40248844601BC604700BFF9A6000086
:103FB00001B40248844601BC604700BF05340100DB
:103FC00001B40248844601BC604700BF851201006D
:103FD00001B40248844601BC604700BF75F8000088
:103FE00001B40248844601BC604700BFA96F0100CC
:103FF00001B40248844601BC604700BF21A900000B
:1040000001B40248844601BC604700BF214400005F
:1040100001B40248844601BC604700BFCD0C0100DA
:1040200001B40248844601BC604700BF91380011CA
:1040300001B40248844601BC604700BF018900000A
:1040400001B40248844601BC604700BFBD5C01006A
:1040500001B40248844601BC604700BF2D6C0100DA
:1040600001B40248844601BC604700BFADAE000009
:1040700001B40248844601BC604700BF85C100000E
:1040800001B40248844601BC604700BFF535010019
:1040900001B40248844601BC604700BF01340100FE
:1040A00001B40248844601BC604700BF3D71010075
:1040B00001B40248844601BC604700BF0D520100B4
:1040C00001B40248844601BC604700BFC56D0100D1
:1040D00001B40248844601BC604700BFF9ED00000E
:1040E00001B40248844601BC604700BFE9170100E3
:1040F00001B40248844601BC604700BFC1F700001C
:1041000001B40248844601BC604700BFE5A000112D
:1041100001B40248844601BC604700BF01D70000DB
:1041200001B40248844601BC604700BF19FA000090
:1041300001B40248844601BC604700BFE9D40000D6
:1041400001B40248844601BC604700BFED6B01002A
:1041500001B40248844601BC604700BF090E00005C
:1041600001B40248844601BC604700BF71B0000042
:1041700001B40248844601BC604700BF51B800004A
:1041800001B40248844601BC604700BFB70E00007E
:1041900001B40248844601BC604700BF8D82000024
:1041A00001B40248844601BC604700BF7997000013
:1041B00001B40248844601BC604700BFD9B000008A
:1041C00001B40248844601BC604700BF9DA90000BD
:1041D00001B40248844601BC604700BF8914010055
:1041E00001B40248844601BC604700BF8B52010005
:1041F00001B40248844601BC604700BF016C010065
:1042000001B40248844601BC604700BFEDA5000030
:1042100001B40248844601BC604700BFF935010083
:1042200001B40248844601BC604700BFE94C01006C
:1042300001B40248844601BC604700BFE9F60000B3
:1042400001B40248844601BC604700BFD544010068
:1042500001B40248844601BC604700BFE51201007A
:104260000200000042BE001101000000F8BB001176
:10427000020000003EBE001101000000A042FF1F2E
:104280000200000000BC001101000000A863FF1F35
:10429000020000003CBE0011030000001C63FF1F71
:1042A000120000000200000042BE001101000000E8
:1042B00040BC0011020000003EBE001101000000E1
:1042C0003DBC0011020000004ABC001103000000C8
:1042D0005763FF1F020000003CBE001103000000F6
:1042E0006C63FF1F020000003EBE001101000000D1
:1042F0003CBC00110200000048BC0011030000009B
:104300002D63FF1F020000003CBE001103000000EF
:104310004E63FF1F0200000042BE001101000000BA
:1043200080BC0011020000003EBE00110100000030
:10433000E943FF1F0200000092BC001101000000D1
:104340007BBC0011020000003EBE00110100000015
:10435000E843FF1F0200000090BC001101000000B4
:104360007463FF1F020000003EBE00110100000048
:10437000E743FF1F020000008EBC00110100000097
:104380006BBC0011020000003EBE001101000000E5
:10439000E643FF1F020000008CBC0011010000007A
:1043A00066BC0011020000003EBE001101000000CA
:1043B000E543FF1F020000008ABC0011010000005D
:1043C00061BC0011020000003EBE001101000000AF
:1043D000E443FF1F0200000088BC00110100000040
:1043E0005CBC00110202020202020000A94A001194
:1043F000A74A0011D4BC0011900118001800FFFF5B
:104400000701020304050602010600000000000087
:10441000000000000000000000000000000000009C
:1044200000000000000003000200000042BE001176
:104430000100000054BD0011020000003EBE00114A
:10444000010000009844FF1F020000005EBD001143
:1044500001000000A263FF1F020000003CBE00112B
:10446000030000001066FF1F020000003EBE0011A6
:10447000010000009844FF1F020000005CBD001115
:1044800001000000A463FF1F020000003CBE0011F9
:10449000030000000866FF1F12A6A6A60000000089
:1044A0000001000000000111FFFF000050485936D4
:1044B000000000000000000001000000E5BC001149
:1044C0000B000500F7000000B400002800280028B9
:1044D0003075A000A000A000A00000080008E001C6
:1044E000F00010001000100010001000100050002C
:1044F0005000500010001000D00700000000000025
:104500000F0001000500307507001000010081FF59
:1045100000000000FF000000BD720011C570001116
:10452000556E0011FFFF0100FF000000D99C001133
:10453000559A00116D990011000000000000000064
:1045400000000800040000003B0001085902E001DF
:1045500088212800FF0000000200000042BE001178
:104560000100000008BF0011020000003EBE001163
:1045700001000000D545FF1F020000003ABE0011F7
:1045800001000000246AFF1F020000003EBE00116F
:1045900001000000D445FF1F0200000038BE0011DA
:1045A00001000000D245FF1F020000003EBE0011C6
:1045B00001000000D045FF1F0200000036BE0011C0
:1045C00001000000C845FF1F1800180000009001FE
:1045D00002000003020200000200000042BE0011BF
:1045E000010000001CBF0011020000003EBE0011CF
:1045F000010000001846FF1F0200000034BE001139
:104600000000000000000000020000003CBE00119D
:0A46100003000000446AFF1F20FFB2
:040000051FFF184180
:00000001FF
